:100000000C940B030C9428030C9428030C942803E1
:100010000C9428030C9428030C9428030C945F324E
:100020000C9428030C9428030C9438280C94F4277F
:100030000C9435290C9428030C9428030C94280361
:100040000C9428030C9428030C9428030C94280384
:100050000C9428030C9411290C9428030C94280365
:100060000C9428030C9428030C9428030C94280364
:100070000C9428030C9428030C9428030C94280354
:100080000C9428030C9428030C9428030C94280344
:100090000C9428030C9428030C9428030C94280334
:1000A0000C9428030C9428030C94280305010902DE
:1000B000A10185020901A1000509190129081500FE
:1000C0002501950875018102050109300931158165
:1000D000257F95027508810609381581257F9501D0
:1000E00075088106050C0A38021581257F95017572
:1000F000088106C0C005010980A101850319012AF4
:10010000B700150126B700950175108100C0050CD8
:100110000901A101850419012AA002150126A002E6
:10012000950175108100C00660FF0961A101096297
:10013000150026FF00952075088102096315002629
:10014000FF00952075089102C005010906A101056F
:100150000719E029E7150025019508750181029529
:1001600001750881010507190029FF150026FF0008
:100170009506750881000508190129051500250156
:10018000950575019102950175039101C0FD377ABE
:10019000585A000004E6D6B44602002101160000B9
:1001A00000742FE5A3E004AE01565D003D8889860A
:1001B000D3DC0AE842C324925842588FD8E75CA0A7
:1001C000D2616E26E888019A676C7887BC8D370902
:1001D000E9D5B739F4E81FA1588DAC1F8AD1B231E7
:1001E000310947F61CBFFFD9CCDFA7E34854EDF532
:1001F000D1109FD138BC29FCFF64C31636C878D40F
:10020000C49AAFCF36FD05742F195A7D842EA19C58
:10021000DF98E88625C64F0A607B98F5AD985CC7E5
:10022000B01AAB783D4FFF5809AF5A1590FECB502E
:10023000804F11BF6EBB6058C7CEA8ED87E4DF8C3E
:100240007F0461157CE3A2DB0E4AD173460C94E96E
:1002500067C597BE8EA3966DAAE8D2CD55A13ECDB7
:1002600058FBAAAEC8DD456C3999DDACB41B1C0B3C
:100270005ACBF899D933014C65216E2195CD6A2E60
:100280008B8E0DBF9F49F1ACBDFED4560F86817495
:1002900026F8EA663F54576D9571BD521BDD384D07
:1002A000AF4D46EAD53F9446DB882BABFDD4064CD8
:1002B00093CBD0EF48F0F93CE6F74C2EEFBE4CCF95
:1002C0002FDBAF761829DDB622EB6DB3EEB22DBC75
:1002D0003F41D54CC08FA535C599D8FB873F95AA1E
:1002E00039F24BF32B455C80F80AC85E972B3A1C19
:1002F000097D3057D1A8F88982D625FF4D2549219F
:100300005300000000CA4E3964D90BC0B80001F296
:1003100002AF090000730D16FBB1C467FB020000B9
:10032000000004595A010001009E04DC0DC10D00BB
:1003300000020002009A04DC0DC10D000003000160
:10034000009F04DC0DC10D0000040002008404DCE9
:100350000DC10D9A0705000100A004DC0DC10D00C0
:1003600000060002008604DC0DC10D00000700023B
:10037000009C04DC0DC10D000008000100A104DC9C
:100380000DC10D0000090002008804DC0DC10D75CF
:10039000070A0002008A04DC0DC10D75070B00027C
:1003A000008C04DC0DC10D75070C0002008E04DC0E
:1003B0000DC10D75070D0002009004DC0DC10D7517
:1003C000070E0002009204DC0DC10D75070F00023C
:1003D000009404DC0DC10D7507100002009604DCCA
:1003E0000DC10D7507110002009804DC0DC10D75DB
:1003F0000712000200A204DC0DC10D000013000270
:1004000000A404DC0DC10D000014000100A604DCF2
:100410000DC10D0000150000000000FB06A1150035
:1004200000290014000F0018003600370000002BD0
:100430000008000C00040012002D0000000000E184
:10044000001D001B0006001900000000000000E273
:1004500000E300E0002800000000000000000000B1
:1004600000000000002C0009001A0015001C0038D4
:1004700000330000000E001700110016000B0013DF
:100480000000000A00070010000D00050000000039
:10049000002A00E400E700E600000000000000522F
:1004A00000500051004F0028000000000009025BCE
:1004B00000030100A0FA0904000001030101000982
:1004C00021110100012244000705810308000109F0
:1004D0000401000203000000092111010001222291
:1004E000000705820320000107050303200001091E
:1004F0000402000103000000092111010001227B18
:10050000000705840320000112010002000000081A
:10051000EDFE00000001010203011C0376006900EA
:1005200061006C003A00660036003400630032005F
:1005300062003300630000000E0370006F0074005F
:100540006900340038000000180373006800690077
:100550006200610064006F0067006300610070006A
:100560000000040309040000000000000000000077
:10057000000000000000000000000000000000007B
:10058000000000000000000000007E0F00D4FFFF0C
:10059000FFC70000007800000000000000002A2BC8
:1005A0002800000000000000000000000000000023
:1005B0000029000000002C1E34202122243426278C
:1005C000252E362D3738271E1F20212223242526AD
:1005D0003333362E37381F0405060708090A0B0C7B
:1005E0000D0E0F101112131415161718191A1B1CC3
:1005F0001D2F3130232D350405060708090A0B0C81
:100600000D0E0F101112131415161718191A1B1CA2
:100610001D2F3130354C11241FBECFEFDAE0DEBF85
:10062000CDBF11E0A0E0B1E0E8E4F9E602C005903A
:100630000D92AC39B107D9F725E0ACE9B1E001C0C2
:100640001D92A532B207E1F70E945C290C94773421
:100650000C940000482F209123059091DA0459E072
:10066000291302C080E0089530E0529FF001539FAB
:10067000F00D1124E552FB4F8181681306C0808183
:10068000481303C085818111EECF2F5F3F4F277044
:10069000E7CFFC01AC014B5F5F4F8FEF91E32191FE
:1006A000822728E030E087FF09C0880F8927215082
:1006B0003109C9F7E417F50791F70895880FF7CFC7
:1006C000E8EDF0E080818E7F80831092E20010924E
:1006D000DA001092E100A0EEB0E08C9181608C9382
:1006E00080818F77808319BCA7EDB0E08C918E7FDD
:1006F0008C9380818F7E80831092C3040895209113
:10070000E4003091E50095E6A9012091EC00822FEC
:10071000817020FF06C08091E80080FF06C080E065
:1007200008952091E80022FD1AC08091D00488230A
:1007300089F0853089F08091EB0085FD0FC0209114
:10074000E4003091E50042175307F9F29150E1F6C9
:1007500084E0089582E0089583E0089581E008959B
:100760008091D20487FF13C08091E80082FF06C009
:100770008091E8008B778093E80004C08091D004DA
:100780008111F2CF08958091D0048823D9F380910C
:10079000E80080FFF8CF8091E8008E77ECCF982FAB
:1007A0009093E900242F762F50E0891731F0709153
:1007B000EC002091ED005091F00021FD07C09F5FFB
:1007C000973071F78093E90081E008953091EB0054
:1007D0003E7F3093EB003091ED003D7F3093ED0094
:1007E0003091EB0031603093EB007093EC0020937C
:1007F000ED005093F0002091EE0027FDE0CF80E067
:100800000895B0E0A0E0E7E0F4E00C948533C8ED93
:10081000D0E088818F7E8883E7EDF0E08081816081
:10082000808384E082BF81E08093C30488818E7FCF
:10083000888302EE10E0F80110821092DA0081EE57
:10084000C82ED12CF601108288818F778883888109
:100850008068888388818F7D888319BC1092D0043A
:100860001092D1041092CF041092CE0490EEE92E93
:10087000F12CF70180818B7F808388818160888360
:1008800042E060E080E00E94CF03F60180818E7F2D
:100890008083F8018081816080838081886080838B
:1008A000F70180818E7F8083888180618883CDB7C6
:1008B000DEB7E8E00C94A133FC018091D80490915C
:1008C000D90486179707A0F06115710529F4909156
:1008D000E8009E779093E80090E06115710551F46F
:1008E000911108C08091E80082FF34C080E0089533
:1008F000BC01F2CF8091D0048823C1F18530C1F1D1
:100900008091E80083FD30C08091E80082FDEACF4D
:100910008091E80080FFE1CF8091F3002091F20008
:10092000382F6115710519F02830310558F091E024
:100930002830310509F090E02091E8002E772093CF
:10094000E800CBCF81918093F100615071092F5F56
:100950003F4FE7CF8091D004882341F0853041F0AC
:100960008091E80083FFBECF81E0089582E0089582
:1009700083E0089508958091C504089587E797E777
:10098000909301088093000888E19AE00FB6F894EC
:10099000A895809360000FBE90936000FFCF9C01EC
:1009A0004FB7F8948091BF049091C004A091C10406
:1009B000B091C2044FBF821B930B08952FB7F894D8
:1009C0006091BF047091C0048091C1049091C204F1
:1009D0002FBF08952FB7F8948091BF049091C00461
:1009E000A091C104B091C2042FBF0895E0EAF1E0E4
:1009F0009191891303C0DF0111971C9291E0E63AAF
:100A0000F907B1F708959C01FC0132969FEF80E051
:100A10004191461751F09F3F19F4411101C0982FA1
:100A20008F5F8630A9F79F3F09F40895290F311D84
:100A300097FD3A95F90162830895A3E0B0E0E3E2FF
:100A4000F5E00C948B332091BC043091BD04281741
:100A50003907A1F09093BD048093BC04E091BA04DF
:100A6000F091BB04309751F024E029839B838A8363
:100A70000084F185E02DCE01019609952396E2E0F0
:100A80000C94A733A3E0B0E0E8E4F5E00C948B33DA
:100A90002091B8043091B90428173907A1F0909338
:100AA000B9048093B804E091BA04F091BB04309784
:100AB00051F023E029839B838A830084F185E02D14
:100AC000CE01019609952396E2E00C94A73380911C
:100AD000B604882359F0E091BA04F091BB04309732
:100AE00029F00190F081E02D0995089580E00895A6
:100AF0004115510511F0FA01099508950E94EA0483
:100B00009C019091B0048091B104982B21F0309316
:100B1000AD042093AC049091B2048091B304982B5F
:100B200021F03093AB042093AA04E091BA04F09131
:100B3000BB04309749F082E08093AE040680F781D1
:100B4000E02D8EEA94E0099508958091A90480FF34
:100B50000CC060913B0170E0759567957595679540
:100B60006115710549F1862F089581FF06C06091D6
:100B70003B0170E075956795F3CF60913B0182FD75
:100B80000BC09091A8049923A1F060913A01809143
:100B90003B01961738F0682F70E06038710500F35C
:100BA0008FE70895899FC001112470E00E94C63329
:100BB000F4CF61E070E0D7CF81E008958091A9047F
:100BC00060918C0470918D0480FF16C020913901D2
:100BD000269FC001279F900D1124BC017695679533
:100BE000769567956038710508F043C06115710509
:100BF00009F441C0862F089581FF0BC0209139016F
:100C0000269FC001279F900D1124BC017695679502
:100C1000E9CF82FF09C0809139019B01829FB00119
:100C2000839F700D1124DECF209183042223D1F203
:100C30009091380180913901482F50E0291748F0F0
:100C4000CB01849FB001859F700D949F700D11247E
:100C5000C9CF289F90011124269FA001279F500DE6
:100C6000369F500D1124692F70E0CA010E94B233E3
:100C7000B9CF8FE7089581E00895282F35EB23033E
:100C8000C001112497FF04C080589109892F08954D
:100C900080589F4FFBCFCF93DF93EC0140917804B6
:100CA0005091790460917A0470917B042FB7F89485
:100CB0008091BF049091C004A091C104B091C2047E
:100CC0002FBF841B950BA60BB70B843F9140A1054A
:100CD000B10518F58091780490917904A0917A0477
:100CE000B0917B048093740490937504A093760470
:100CF000B093770484EF91E0A0E0B0E080937004BB
:100D000090937104A0937204B0937304D093800401
:100D1000C0937F04DF91CF9108950E94DE04609319
:100D2000740470937504809376049093770482E33F
:100D300090E0A0E0B0E0E2CFFC018481862351F492
:100D400092819923B9F06923808583FF05C081E0F2
:100D500061110FC080E00895892F8F7092959F7068
:100D6000982B862F8F7062956F70682B81E0961399
:100D7000F1CF089581E0FDCFDC0160916A0480919C
:100D80006B04962F891301C00895292F30E0F901D3
:100D9000EE0FFF1FEE59FB4F408151814A175B0751
:100DA000A1F487E08A9FA0018B9F500D11244F531F
:100DB0005C4F81E0FA0184839613E6CF2F5F3F4FAB
:100DC0002370332720936A0408952F5F3F4F922F9B
:100DD0009370D8CF1092BF031092BE03E1ECF3E002
:100DE0008581811102C014821682379683E0E93F23
:100DF000F807B1F70895B0E0A0E0E1E0F7E00C9467
:100E000083338FEF9FEF4430510508F469C0409160
:100E1000970341FB882780F990E0880F991F42FBD8
:100E2000002700F910E0000F111F000F111F802B89
:100E3000912B40FBCC24C0F8D12C8C299D2943FB5D
:100E4000222720F9C22FE0E0DE2F53E0CC0FDD1F78
:100E50005A95E1F78C2B9D2B44FBAA27A0F9B0E013
:100E6000E4E0AA0FBB1FEA95E1F78A2B9B2B45FB19
:100E7000EE27E0F9F0E0A5E0EE0FFF1FAA95E1F7FD
:100E80008E2B9F2B46FB222720F930E0B6E0220F65
:100E9000331FBA95E1F7822B932B47FB222720F9CA
:100EA00030E03695322F222737952795822B932BCA
:100EB00020919803322F3170F32EE82EF92A2695CF
:100EC0002170B22EBB0CA82EBF28C501BB0CAA0BEB
:100ED000BB0BFB0180839183A283B38390E080E00E
:100EE000CDB7DEB7EAE00C949F33E4E8F4E0848108
:100EF00095812AE030E0B9010E94B233609333015A
:100F00008681809332018285809339018485809324
:100F1000380186859785B9010E94B233609331010B
:100F2000808980933001828980933B0184898093FA
:100F30003A0108958091840490918504909335013D
:100F4000809334010895EEE4F2E090E080E065E300
:100F500077E24CE557E22BEA36E2778366835187E6
:100F600040873387228797878687019670968830D7
:100F7000910599F7089581152CE7920741F4209186
:100F80006E0430916F04232B11F490E080E00895FB
:100F900080E00895F894E82FE295EF70F0E031A139
:100FA000282F2F7081E090E001C0880F2A95EAF782
:100FB000982F9095932391A392A1892B82A3789443
:100FC00008950F931F938091B604882329F00E94FF
:100FD000DE041F910F9108950E94DE04009101022A
:100FE000109102022091030230910402600F711FE0
:100FF000821F931FEECF811520E59207D0F5811552
:1010000040E4940708F08FC0803E910520F58D3CA8
:10101000910508F080C0883A910578F4853A9105E9
:1010200008F070C08130910519F1009709F1843002
:101030009105F0F490E080E01BC0833C9105D0F76F
:10104000885AE82FF0E0EE0FFF1FEC5AFE4F808128
:10105000918194640895811550E2950708F0B8C015
:10106000811561E0960708F058C0883E910510F799
:101070000895803672E5970720F5803422E59207BF
:1010800008F05BC0803242E5940708F04FC081153C
:1010900052E5950708F483C0282F2695269570E21F
:1010A000279F90011124837041E050E0BA0102C0F3
:1010B000660F771F8A95E2F7CB01822B932B9D68F1
:1010C0000895803A62E5960760F4803872E59707E4
:1010D00008F449C08F7190E0982F8827846F906A38
:1010E0000895803C22E5920708F453C0803E42E513
:1010F000940708F09FCF982F882788279F71806FCB
:10110000906A0895855AE82FF0E0EF5AFE4F8081EB
:1011100090E0906408959065089520E0392FB9011A
:10112000682BCB0108959F70906A08958F7190E0AD
:10113000982F8827816F906A0895282F26952695E5
:10114000277070E2279F90011124837041E050E0E6
:10115000BA0102C0660F771F8A95E2F7CB01822B96
:10116000932B9C680895282F26952695277070E26A
:10117000279F90011124837041E050E0BA0102C022
:10118000660F771F8A95E2F7CB01822B932B9A6823
:1011900008958F7190E0982F8827906208959C01A0
:1011A00095E0369527959A95E1F72F7030E0322F2C
:1011B0002227482F4F7150E084FF05C084E0440F80
:1011C000551F8A95E1F7C901842B952B90690895E5
:1011D0009F71E3CF8091DC01882331F01092DC0114
:1011E0001092DB011092DA010895CF93C82F8091FD
:1011F000980382FF0CC08091DC018C1741F00E94A3
:10120000EA049093DB018093DA01C093DC01CF9173
:1012100008959091DC01292F282361F0809589237E
:101220008093DC01882339F00E94EA049093DB016B
:101230008093DA01089590E080E0F8CF8095909156
:1012400024059823909324050895809590919903FF
:10125000982390939903089590919903892B8093F3
:10126000990308951092D1011092D0011092CF01EC
:1012700008958091860490918704892B89F00E94BB
:10128000EA042091DA013091DB01AC01421B530BDF
:1012900081E020918604309187044217530708F4B7
:1012A00080E0817008959091CE01292F282321F0AC
:1012B000809589238093CE01089580912305909194
:1012C000DA04981301C008958F5F8770FACF292F31
:1012D0009A3078F5873068F590E037E0239F800DED
:1012E000911D1124682F677023E0969587952A95A4
:1012F000E1F7FC01EE0FFF1FE80FF91FE655FE4F67
:1013000050E040E080E0219130E0062E02C03695AA
:1013100027950A94E2F721703327042E01C0220F8B
:101320000A94EAF7822B4F5F5F4F4330510559F71C
:10133000089580E00895292F9A3098F5873088F530
:1013400090E037E0239F800D911D1124282F2770F6
:1013500041E001C0440F2A95EAF723E0969587956E
:101360002A95E1F7FC01EE0FFF1FE80FF91FE65584
:10137000FE4F30E020E070E05191DF011197CB018A
:10138000022E02C0969587950A94E2F781708195A6
:101390008527842385278C932F5F3F4F233031058A
:1013A00059F708958093120208959091120221E056
:1013B00030E0F90101C0EE0F8A95EAF7D90102C0C9
:1013C000AA0FBB1F6A95E2F7EA2B01C0220F4A95CC
:1013D000EAF7892F8E23E81305C0292B822F0E945C
:1013E000D209089520952923F9CF21E030E001C0EA
:1013F000220F8A95EAF720958091120282230E949B
:10140000D20908959091D101809589238093D101CB
:10141000282F277069F4891759F09091980392FF4B
:1014200007C08695869586950E94F5090E94320927
:10143000089521E030E001C0220F8A95EAF78091FB
:101440001202822B0E94D20908959091980392FF74
:1014500010C098E0899F90011124622B6093D10104
:101460000E94190A0E94EA049093D0018093CF0150
:1014700008950E94190A0895809311020895929583
:101480009F70963091F058F4925F9F70923058F4AC
:10149000803F19F030F4883E30F481E008959A5F7F
:1014A000F4CF843FD1F380E00895883EB0F3813FCC
:1014B000D1F7F3CF662309F45DC08D3C41F40E945F
:1014C000DE0581958093B1040E947E0508958E3CCF
:1014D00019F40E94DE05F6CF8F3C31F40E94DE0540
:1014E00081958093B004F0CF803D19F40E94DE0511
:1014F000F8CF893D29F40E94A5058093B204E4CF7A
:101500008A3D21F40E94A5058195F7CF8B3D31F4EA
:101510000E94A50581958093B304D6CF8C3D19F424
:101520000E94A505F8CF9FE2980F983070F4815D76
:10153000990B21E030E001C0220F8A95EAF78091F3
:10154000AF04822B8093AF04BFCF8D3D31F48091E7
:10155000A90481608093A904B7CF8E3D21F48091C6
:10156000A9048260F7CF8F3D09F0AECF8091A90426
:101570008460F0CF4091B0048D3C59F48091B10467
:1015800087FF0DC01092B10441110BC0109283046B
:1015900008C08E3C81F48091B10418169CF344235A
:1015A00081F08091B2049091B304892B09F08CCF23
:1015B0001092A80489CF8F3C49F447FFF0CF1092D6
:1015C000B0048091B1048111ECCFE0CF803D19F4DB
:1015D0001416ACF3E4CF9091B204893D29F41916A6
:1015E000F4F61092B204DBCF8A3D19F497FFD7CFFF
:1015F000F8CF9091B3048B3D29F497FFD0CF109290
:10160000B304CDCF8C3D19F41916CCF3C8CF9FE2AB
:10161000980F983090F4815D990B21E030E0B9018A
:1016200002C0660F771F8A95E2F7CB0180959091F3
:10163000AF0489238093AF04B2CF8D3D31F4809104
:10164000A9048E7F8093A904AACF8E3D21F48091B6
:10165000A9048D7FF7CF8F3D09F0A1CF8091A90418
:101660008B7FF0CF9C013A9521153F4150F5FC014D
:10167000EE27F170BC0166277270AC0144275470EC
:101680009C012227387094FF0EC080E1EF2B09F4F3
:1016900080E0672B09F08062452B09F08064232BE2
:1016A00089F08068089581E0EF2B09F480E0672BD2
:1016B00009F08260452B09F08460232B19F08860C3
:1016C000089580E008950F931F93CF93DF938B01CC
:1016D000EA019091D004943061F58093E9008FEF96
:1016E0009091E800815095FD06C095ED9A95F1F72F
:1016F00000008111F5CF8091E80085FF1AC00E949B
:101700007F03811111C08091E80085FD06C08091A2
:10171000E8008E778093E800F2CFF80181918F0185
:101720008093F100219779F78091E8008E7780937C
:10173000E800DF91CF911F910F91089543E050E0B1
:10174000BC0184E00E94630B089546E050E0BC01B8
:1017500084E00E94630B0895CF93DF93EC0148E08F
:1017600050E0BC0181E00E94630B88E0FE01A6EC22
:10177000B4E001900D928A95E1F7DF91CF91089541
:10178000019708F40895EFE9FFE03197F1F700C001
:101790000000F6CFB0E0A0E0E0EDFBE00C94833376
:1017A0007C015B016A018091000201E010E08A3057
:1017B00010F40AE010E0C1E0D0E0B501C701F60185
:1017C0000995811104C021960C171D072CF4CDB783
:1017D000DEB7EAE00C949F33CC9F9001CD9F300D93
:1017E000300D112490E080E045E34A95F1F70000C8
:1017F000019682179307C1F7E0CFCF93C82F6FEF01
:10180000811164E084E290E00E943B346FEFC111EB
:1018100064EB85E290E00E943B346FEFC1116CEA0B
:1018200086E290E00E943B34CF910895CF93DF93FE
:10183000CCE6D3E060E0CE010E943B342196C11596
:1018400084E0D807B9F7DF91CF9108951F93CF9324
:10185000DF93122F8430E0F46A30D0F44730C0F4C4
:10186000C42FD0E0CC0FDD1F9EE0699FC00DD11DBD
:1018700011249CE8899FC00DD11D1124632FCE0136
:1018800088960E943B34612FCE0189960E943B349A
:10189000DF91CF911F91089584E290E00E941D3462
:1018A000843089F485E290E00E941D34843B59F431
:1018B00086E290E00E941D3491E08C3A09F090E0BD
:1018C000892F8170089580E0FCCF0F931F93CF93F1
:1018D000DF93843030F56A3020F5473010F5C42F9F
:1018E000D0E0CC0FDD1F2EE0629FC00DD11D112472
:1018F0003CE8839FC00DD11D1124CE0188960E9423
:101900001D34082F10E0102F0027CE0189960E9469
:101910001D349801282BC901DF91CF911F910F91A0
:10192000089590E080E0F8CF462F20913802309162
:101930003902232B99F4703F39F4603F79F4809198
:101940003A0290913B0208957A3040F4673030F4C7
:10195000843020F4672F0E94650C089590E080E0A9
:101960000895CF92DF92FF920F931F93CF93DF934F
:101970006C010091120280911102082BC3E0D0E0AB
:1019800010E0FC2EC8010C2E02C0959587950A9494
:10199000E2F780FD0CC02197A0F7F12C8F2DDF918D
:1019A000CF911F910F91FF90DF90CF900895B601D6
:1019B0008C2F0E94940C0E94FB07019761F3EECFDD
:1019C000CF93DF93EC010E94B10CBE010E94940CF6
:1019D0000E94FB07DF91CF910895FC018481882349
:1019E00071F087819085009729F00E94FB070E9483
:1019F0003F0A0895808191810E94E00CF8CF80E039
:101A00000895A6E0B0E0E7E0FDE00C948A33498356
:101A10005A8349815A819923A1F0222391F0CA0166
:101A20000E94B10C182F682F89819A810E949B090E
:101A300069817A81812F0E94940C2696E3E00C94B0
:101A4000A633CA010E946709182FF2CFFC01262F86
:101A500087819085009741F4408151816281738133
:101A6000848195810E94010D08950F931F93CF9358
:101A7000DF9304E814E0C8E5D2E0CE010E941D34F3
:101A8000F80161918F01681719F0CE010E943B3473
:101A90002196CC37F2E0DF0781F7DF91CF911F91DC
:101AA0000F9108950F931F93CF93DF9304E814E0F1
:101AB000C8E5D2E0CE010E941D34F80181938F0168
:101AC0002196CC37F2E0DF07A9F7CFE2D3E0FE01A1
:101AD00085919491009711F0FC0109952C96F4E002
:101AE000CB32DF07A1F7DF91CF911F910F910895BE
:101AF0009B01883070F49AE0899FB00111246458EA
:101B00007D4F4AE050E0C9010E940D3490E080E032
:101B100008958FEF9FEF0895AAE0B0E0E2E9FDE0BD
:101B20000C948B339C0137552F3F310509F068F435
:101B3000BE016F5F7F4F0E94780D892B31F489853C
:101B40009A852A96E2E00C94A73380919C049091A8
:101B50009D04F7CF9091980392FB222720F9281734
:101B600079F080FB92F990939803609197037091BC
:101B7000980384E090E00E94593482E00E94020AB7
:101B80000895DA019C012E5F3F4FF9014591549170
:101B9000F90125913491A217B30758F0FC0134964E
:101BA000859194910E94FD330E94350D90E080E074
:101BB00008958FEF9FEF0895DB01FC013296259188
:101BC00034914217530758F0FC0134966591749193
:101BD000A901CD010E94FD3390E080E008958FEFD0
:101BE0009FEF0895AAE0B0E0E8EFFDE00C948333A6
:101BF0000FE113E08CE1E82E83E0F82E97E0B92E98
:101C00002EE1C22E23E0D22EAA24A3944AE050E073
:101C1000B701CE0101960E940D34F8013896DF011C
:101C20008B2D1D928A95E9F789819A81D8011196A9
:101C30009C938E938F8112968C9312978D8113961D
:101C40008C931397888514968C9314978985159691
:101C50008C9315978B819C8117969C938E931697E6
:101C600018961C9218978A8587FF3CC01E961C9276
:101C70001E921D9780FF03C0D8011896AC9281FF79
:101C800004C0F80190859260908782FF07C0D80158
:101C900018969C911897946018969C9383FF04C0A3
:101CA000F80190859860908784FF07C0D801189646
:101CB0009C911897906118969C9385FF04C0F80139
:101CC000808580628087FAE0EF0EF11C015F1F4F74
:101CD0008CE6E81683E0F80609F098CF2A96EAE049
:101CE0000C949F33F801D686C586C4CFAAE0B0E035
:101CF000ECE7FEE00C948533EEECF2E080E5DF01EA
:101D00001D928A95E9F7E1ECF3E088E3DF011D928B
:101D10008A95E9F78EECC82E82E0D82E7F010CEC74
:101D200012E0F701D182C0824AE050E0B801CE0152
:101D300001960E940D3488E0FE013196D601019093
:101D40000D928A95E1F789859A85D70113969C9320
:101D50008E931297BAE0CB0ED11CE7E0EE0EF11C89
:101D6000065F1F4F0C31F3E01F07D9F62A96E8E013
:101D70000C94A133A4E0B0E0E0ECFEE00C948A33D4
:101D80004091FC015091FD016091FE017091FF01B5
:101D90002FB7F8948091BF049091C004A091C10422
:101DA000B091C2042FBF841B950BA60BB70B11E09B
:101DB00084369105A105B10570F10E94E1076E5FBF
:101DC0007F4F8F4F9F4F69837A838B839C83809152
:101DD0001201909113018E509E4F4091110150E0DD
:101DE0004530510510F044E050E0BE016F5F7F4F79
:101DF0000E94FD3382E090E00E940533182F882373
:101E000051F00E94DE046093FC017093FD01809309
:101E1000FE019093FF01812F2496E3E00C94A633FA
:101E2000EF92FF921F93CF93DF9300D000D000D0AA
:101E3000CDB7DEB77B0190E080E00E940533182F1C
:101E4000882309F46AC04091040150E0411551050E
:101E500011F041E050E060910501709106016E5073
:101E60007E4FCE0106960E94FD334091EE015091C7
:101E7000EF016091F0017091F1012FB7F89480911A
:101E8000BF049091C004A091C104B091C2042FBFBF
:101E9000841B950BA60BB70B84369105A105B105E4
:101EA00038F483EF91E00E9449039E818917A9F1DC
:101EB00081E090E00E940533882309F44EC04091F0
:101EC0000C0150E04630510510F045E050E06091C3
:101ED0000D0170910E016E507E4FCE0101960E9451
:101EE000FD3383EF91E00E9449039E81891335C041
:101EF0000E94DE046093EE017093EF018093F00185
:101F00009093F10185E0FE013196A9EEB1E00190D8
:101F10000D928A95E1F711E00BC085E0E3EFF1E067
:101F2000DE01119601900D928A95E1F71111EACF29
:101F300085E0E9EEF1E0D70101900D928A95E1F795
:101F4000812F26960FB6F894DEBF0FBECDBFDF916E
:101F5000CF911F91FF90EF90089510E0E9CFAFE08F
:101F6000B0E0E5EBFFE00C9480338E010F5F1F4F74
:101F70008AE0F80111928A95E9F780E2C82E81E0A3
:101F8000D82EF12CE12CAA24A394B12C20E2822E8D
:101F900021E0922EF60181916F018F3F09F442C03A
:101FA000F894E82FE295EF70F0E021A18F70A50181
:101FB00002C0440F551F8A95E2F7CA01922F982B51
:101FC00091A392A18095892382A3789400C0E9E12E
:101FD000F1E0712C31E021912F3F09F48CC0A22F48
:101FE000A295AF70B0E090968C9190E02F7002C0F7
:101FF000959587952A95E2F780FD7DC0832F782AF5
:10200000330F8E169F0639F7F601319780818F3F87
:1020100011F00E94CA0750EA5A95F1F7F801EE0D47
:10202000FF1D70828FEFE81AF80AE5E0EE16F10462
:1020300009F0B0CF4AE050E0B80185E092E00E949C
:10204000F033009741F02AE0F801A5E0B2E00190FA
:102050000D922A95E1F70091100210E0025D1D4FEC
:10206000892B09F44AC081E08093E1010E94EA04CF
:102070009093E0018093DF01F12CE090B604EE2014
:1020800009F492C06E01FBE0CF0ED11C85E0F60191
:1020900011928A95E9F7809100028A3008F051C0C8
:1020A00040E15FE0B601C8010E94CA0B882309F431
:1020B0006AC04AEB5EE0B601C8010E94CA0B8823E1
:1020C00009F461C01092000280910F0290E045E097
:1020D00050E0B601825D9D4F0E94F03321E02093D5
:1020E000E801892B09F042C0E12C8E2D8F292F9613
:1020F000EDE00C949C3380E082CFF090E101FF2072
:1021000009F4BACF8091DF019091E0010E94CF04E1
:10211000059708F4B1CF45E050E065E072E0C801F2
:102120000E94F033892B59F085E0E5E0F2E0D80118
:1021300001900D928A95E1F71092E1019ECFF12C6A
:10214000FBCF8091E2019091E3010E94CF04843F94
:10215000914008F0A5CF8091E801882329F285E01D
:10216000F60111928A95E9F71092E801A0910F0209
:10217000B0E0A25DBD4F85E0FE013B9601900D925F
:102180008A95E1F7B2CF809100028F3F31F08F5FE7
:10219000809300028A3008F497CF0E94EA0490935B
:1021A000E3018093E201D7CF85E0F801A3EFB1E02E
:1021B00001900D928A95E1F783EF91E00E94490327
:1021C0008093F2018090F8019090F901A090FA01BB
:1021D000B090FB018091E4019091E501A091E601AE
:1021E000B091E70188169906AA06BB0609F47DCFCF
:1021F0008092E4019092E501A092E601B092E7019D
:102200000E94DE04861A970AA80AB90A809201027F
:1022100090920202A0920302B092040266CFCF9382
:1022200080919903C0912405C82B8091DC018823FB
:10223000E9F08091860490918704892B29F00E940F
:10224000390981110E94EA088091DC01C82B20E045
:1022500080EA91E0FC013191CF0131112F5FF1E073
:10226000863A9F07B9F721110E94EA0880917C0401
:1022700080958C2390917D04892B80939E0148E06A
:1022800050E062ED71E08EE991E00E94F033892B1D
:10229000A9F088E0EEE9F1E0A2EDB1E001900D9245
:1022A0008A95E1F7E091BA04F091BB04309731F0E0
:1022B0000280F381E02D8EE991E00995CF91089598
:1022C000CF93DF93EC014A855B856E857F850E9405
:1022D00078058B810E941E098C810E9425090E942D
:1022E0000F1186E0FE0111928A95E9F7DF91CF91F7
:1022F0000895CF93DF93EC018D8181FD14C082603E
:102300008D83809124059B81892B809324058C816A
:102310000E942C090E940F11488559856E857F8582
:10232000CE010E9478051092B5041092B4048D81FC
:1023300080FD03C0CE010E946011DF91CF9108950E
:1023400080913601877F8093360182E00E941E09CA
:102350008091360184FF06C08F7E8093360182E033
:102360000E942C098091360185FF06C08F7D8093E5
:10237000360180E20E942C090E940F110895CF932C
:1023800010929903C6E0E0EAF1E0DF018C2F1D9284
:102390008A95E9F790E080E00E94420590E080E0B5
:1023A0000E941D05109224050E940F11EEEAF4E030
:1023B000DF011D92CA95E9F7109283041092A804D8
:1023C0001092A9040E947E05CF910895AAE2B0E080
:1023D000ECEEF1E10C948A3382ED94E02091F1006F
:1023E000DC012D93CD01B4E08A3D9B07B9F78091C4
:1023F000D304833009F472C0B8F4813009F449C0C1
:10240000823009F4B3C08091E80083FF96C28091C6
:10241000D2049091D3049A3008F08FC2E92FF0E0F3
:10242000E758FB4C0C94DA338A3009F48EC08B30B9
:1024300009F471C0893039F78091D204813219F7DB
:102440008091D6049091D704009711F00297D9F6A5
:102450008091E800877F8093E8008091E80082FF08
:1024600038C09091F3008091F200029731F480918E
:10247000F100813011F0863021F48091F1008093D9
:10248000C5048091E8008B778093E8000E94B00338
:10249000BACF8091D204813A09F0B5CF8091E8009B
:1024A000877F8093E8008091D6049091D704892B90
:1024B00061F468E086EC94E070E00E945C04809136
:1024C000E8008B778093E8009ECF60E090E080E0AA
:1024D000F3CF8091D0048111C0CF95CF8091D204E9
:1024E000813A09F090CF8091D6049091D704892B3E
:1024F00009F089CF8091E800877F8093E800809180
:10250000E80080FFFCCF80913C018093F100809136
:10251000E8008E77B9CF8091D204813209F073CF71
:102520008091D6049091D704892B09F06CCF8091CB
:10253000E800877F8093E8000E94B0038091D40474
:1025400080933C010E94BF115ECF8091D204813202
:1025500009F059CF8091E800877F8093E8000E94BE
:10256000B0038091D5048093C4044DCF8091D204F0
:10257000813A09F048CF8091E800877F8093E80096
:102580008091E80080FFFCCF8091C404BECF8038EA
:1025900099F0823809F0D1C18091D6048F708730CC
:1025A00008F0CBC18093E9008091EB0085FB882780
:1025B00080F91092E90006C08091CE049091CF047A
:1025C000911182609091E800977F9093E80080934A
:1025D000F1001092F1008091E8008E77AAC1882363
:1025E00009F498C1823009F0A8C18091D404811106
:1025F0009BC18091D6048F702FEF280F263008F0F2
:102600009CC18093E9002091EB0020FF8DC19330A5
:1026100031F48091EB0080628093EB0085C1909152
:10262000EB0090619093EB0021E030E001C0220FBD
:102630008A95EAF72093EA001092EA008091EB0075
:102640008860EACF811179C11091D4041F778091FD
:10265000E3008078812B8093E3008091E800877FFE
:102660008093E8000E94B0038091E80080FFFCCFD7
:102670008091E30080688093E30082E0111183E0A1
:102680008093D0045AC18058823008F056C12091FE
:10269000D4043091D5042C3DE3E03E07A1F583E05E
:1026A0008A838AE289834FB7F894DE01139620E08B
:1026B0003EE051E2E32FF0E050935700E49120FF19
:1026C00003C0E295EF703F5FEF708E2F90E0EA302D
:1026D000C0F0C7968D939D932F5F243159F74FBF5C
:1026E0008091E800877F8093E8006AE270E0CE0185
:1026F00001960E945C048091E8008B778093E8004B
:102700001CC1C096E7CF8091D6049091D704432F87
:1027100055274330510509F44AC078F54130510539
:1027200009F485C08BE590E0EDEAF4E04230510514
:1027300009F003C12091E800277F2093E800209151
:10274000D8043091D9048217930708F49C0140E023
:102750002115310509F070C041116EC08091E8006B
:1027600082FDC9CF8091D004882329F2853019F2E7
:102770008091E80083FFF2CFBECF4132510509F4CA
:1027800047C04232510509F0D8C08330910508F0A6
:10279000D4C0FC01EE0FFF1FE157FE4F0190F08106
:1027A000E02D84579E4FDC018C9190E01DC03327B3
:1027B00021303105E9F02115310579F0223031055C
:1027C000F9F02330310509F0B8C0EAE1F5E0E49111
:1027D0008E2F90E0EAE1F5E007C0E2E6F5E0E49153
:1027E0008E2F90E0E2E6F5E0009709F4A6C0A2CFB4
:1027F000E8E4F5E0E4918E2F90E0E8E4F5E0F4CF32
:10280000E8E3F5E0E4918E2F90E0E8E3F5E0ECCF2B
:102810008330910508F091C0880F991FFC01EB5699
:10282000FE4F0190F081E02D89E090E083CF82E1BE
:1028300090E0E8E0F5E07ECF8091D004882309F4B1
:102840005ACF853009F457CF8091E80083FD53CFEC
:102850008091E80082FD82CF8091E80080FF78CFF0
:102860009091F3008091F2002115310519F0883024
:10287000910550F041E0089709F040E08091E800B0
:102880008E778093E80064CF44914093F1003196B5
:10289000215031090196E8CF803809F04EC080916F
:1028A000E800877F8093E8008091D1048093F10055
:1028B00092CE811142C01091D4041230F0F5809173
:1028C000E800877F8093E8001093D1040E94B00352
:1028D000112311F084E005C08091E30087FDFACF59
:1028E00081E08093D00442E061EC81E00E94CF035C
:1028F00042E261EC84E00E94CF0342E261EC82E0BC
:102900000E94CF0342E260EC83E00E94CF038091FB
:10291000D00413C08091D404813079F481E09330E5
:1029200009F080E08093CF041092E9008091E800E4
:10293000877F8093E8000E94B0038091E80083FFC6
:102940000AC08091E800877F8093E8008091EB00C7
:1029500080628093EB00AA96E3E00C94A633E4E84F
:10296000F4E0128E138E8FEA90E09183808325E04D
:10297000248F88E893E1938382838AE090E09583B3
:10298000848344E150E05783468348E050E0518718
:102990004087938782876EE170E0758764879787A9
:1029A000868780E590E0918B808B538B428B48E249
:1029B00050E0558B448B42E350E0578B468B48ECFC
:1029C00050E0518F408F158E178E168E91A380A3E5
:1029D00022A30E94350D0E94BF11109298031092FD
:1029E0009703E8E9F3E08081846080836091970336
:1029F0007091980384E090E00E9459340E94520D37
:102A00000895AEE1B0E0E7E0F5E10C948333E090A7
:102A10006E04F0906F0481E090E090936F048093D7
:102A20006E04B12C81E2C82E84E0D82EA12C1DC0EA
:102A3000402F21E030E0B11008C0F801EE0FFF1F79
:102A4000EC0DFD1D859194919C016A2D8B2D0E94AA
:102A5000260C0F5F1F4F0730110551F7A3948EE02E
:102A6000C80ED11CEAE0AE1619F010E000E0E0CF8D
:102A7000B394F4E0BF12D6CF0E94AF141A82198229
:102A80001C821B821E821D8218861F8288EC90E0A9
:102A90009A8789870CE712E04AE050E0B801CE013E
:102AA00001960E945F34065F1F4F0C3C82E01807BE
:102AB00099F76E01EBE0CE0ED11C8AE0F60111927F
:102AC0008A95E9F74AE050E0B801C6010E945F34F8
:102AD000065F1F4F0C31F3E01F07A1F76E0185E180
:102AE000C80ED11C8AE0F60111928A95E9F78FEFA2
:102AF0009FEF9A8F898F87E08E8F4AE050E0B80170
:102B0000C6010E945F34065F1F4F0C36F3E01F07BB
:102B1000A1F7F0926F04E0926E046E96EAE00C94D6
:102B20009F3380E00E94FD0B60E087E290E00E940E
:102B30003B340E9401150E94160C81E00E94FD0B9F
:102B40000895CF92DF92EF92FF928FEF9FEF443084
:102B5000510508F46CC0FB01C080D180E280F38095
:102B60000E94BF1180919703C0FA80F9B701A601B6
:102B7000769567955795479540FB81F9B701A60172
:102B800022E076956795579547952A95D1F740FBB2
:102B900082F9B701A60133E0769567955795479579
:102BA0003A95D1F740FB83F9B701A601E4E07695A9
:102BB000679557954795EA95D1F740FB84F9B7019A
:102BC000A601F5E07695679557954795FA95D1F763
:102BD00040FB85F9B701A601A6E076956795579564
:102BE0004795AA95D1F740FB86F9B701A601B7E052
:102BF0007695679557954795BA95D1F740FB87F934
:102C00008093970380919803D0FA80F9D1FACC246D
:102C1000C0F8C0FA81F9809398036091970370918E
:102C2000980384E090E00E94593490E080E0FF90A7
:102C3000EF90DF90CF9008950E94BF112FEF84E3B3
:102C40009CE0215080409040E1F700C0000088E106
:102C50009AE00FB6F894A895809360000FBE909309
:102C60006000FFCF882321F00E941E090E940F11EF
:102C70000895882339F090912405982B909324058A
:102C80000E940F110895882321F00E9425090E94B7
:102C90000F110895882321F00E942C090E940F1122
:102CA0000895882381F19CEF980F913A28F40E94AF
:102CB000F6040E940F11089590E2980F983050F496
:102CC000877091E001C0990F8A95EAF7892F0E94D9
:102CD0002509EFCF9BE5980F933028F490E080E032
:102CE0000E944205089598E5980F9B3128F490E0E2
:102CF00080E00E941D05089593E3980F933118F426
:102D000060E00E945A0A0895FF920F931F93CF9399
:102D1000DF93F82E009181041091820401151105B2
:102D200009F449C01092800410927F0410927C0430
:102D300010927D04D8011696CD91DC919E013A95B2
:102D400021153F4108F4D07ED1E0C11101C0D0E08F
:102D5000D8011996ED91FC911A97309731F01B9696
:102D60006D917C9180E00995D823DD2339F08CEFBB
:102D70008C0F813A30F58C2F0E94F604FF2099F0D9
:102D8000E0918104F0918204808584FD0CC08091E3
:102D90007E04882341F0808191819C01215031097A
:102DA0002F333E47A0F00E940F1110928204109220
:102DB000810410927E04C801CDB7DEB7E5E00C9423
:102DC000A4330E940F118C2F0E945116D7CF0E945E
:102DD0004B06E9CFCF93DF93EC010E945116CE0151
:102DE0000E94320B9E01205E31092830310510F01F
:102DF000CD2B29F40E944316DF91CF9108950E94B4
:102E00003216FACFCF93C82F8823A1F08CEF8C0F06
:102E1000813A90F4E0EAF1E08191C817E9F181E0AC
:102E2000E63AF807C9F76C2F8EE991E00E94030596
:102E30000E940F11CF91089580E28C0F883048F4E2
:102E4000C77081E001C0880FCA95EAF70E942C097B
:102E5000EFCFEBE5EC0FE33040F4F0E0EF5AFE4F3C
:102E6000808190E00E944205E5CFE8E5EC0FEB3170
:102E700050F4F0E0EE0FFF1FEC5AFE4F808191817D
:102E80000E941D05D7CF83E38C0F833198F661E054
:102E90008C2F0E945A0ACECF8C2F0E94F6040E94DB
:102EA0000F11C1CF1F93CF93DF93182FEB010E9417
:102EB0000217209739F4812F0E945116DF91CF918C
:102EC0001F9108958FE99FE00197F1F700C000007E
:102ED0002197EFCF6091A4047091A504893321F06C
:102EE0006091A2047091A3040E9452170895B0E06B
:102EF000A0E0EDE7F7E10C948333EC018AE0A82E23
:102F00002881222309F49EC0213009F043C0898121
:102F1000813049F48E010E5F1F4F8A810E946A172B
:102F2000E8012196EDCF823039F48E010E5F1F4FFC
:102F30008A810E940217F4CF833039F48E010E5F2C
:102F40001F4F8A810E945116EBCF843011F02196D9
:102F5000E8CF2A81229690E080E0AE014F5F5F4F7C
:102F60002053330B2A30310550F00097D1F2EFE9AE
:102F7000FFE03197F1F700C000000197F6CFA89E5F
:102F8000B001A99E700D1124C901860F971F2981D8
:102F9000EA01E3CFE22FF0E0EA56FA4FB490822F35
:102FA00086958695869590E0FC01EA57FA4FE49065
:102FB0002770F12C022E02C0F594E7940A94E2F7F0
:102FC000F1E0EF22FF24FC01EA58FA4FC490D12C23
:102FD000022E02C0D594C7940A94E2F731E0C322CE
:102FE000DD24FC01EA59FA4F049110E002C0159566
:102FF00007952A95E2F701701127E114F10419F001
:1030000081EE0E940217C114D10419F086EE0E94CD
:10301000021770E060E08B2D0E945217C114D1049A
:1030200019F086EE0E945116E114F10419F081EEB8
:103030000E9451160115110509F473CF8CE20E940C
:103040006A176FCFCDB7DEB7EAE00C949F33CF930A
:10305000DF93EC010E94320B9E01205E3109283083
:10306000310510F0209741F40E944A168C2F0E94DF
:103070000217DF91CF9108950E943916F7CF66238A
:1030800029F0209124052260209324059C013052D0
:103090002115304308F499270E9427180895B0E0BD
:1030A000A0E0E5E5F8E10C9485336C018B01E42E9A
:1030B0008091360182FF87C0C091BC03D091BD03CF
:1030C000CC15DD0521F0C114D10409F07CC080913C
:1030D00036018B7F8093360181FD6EC08091BA03EB
:1030E0009091BB03A801481B590B81E0209134014A
:1030F000309135014217530708F480E08170F82EB3
:1031000080913601F0FA81F980933601FE0183E067
:10311000F695E7958A95E1F7EE71FF27E656FC4FA5
:1031200020813181AE014F70552781E090E002C0CF
:10313000880F991F4A95E2F7FF2009F43FC0822BC0
:10314000932B918380838091990381FF08C08091A4
:10315000360180618093360182E00E9425098091CA
:10316000990385FF08C08091360180628093360103
:1031700080E20E9425096F2DCE010E943F18EE20AB
:1031800031F080919F0485FF02C086FF30C080919E
:10319000A2049091A3040E94C00B8091BC03909163
:1031A000BD039C0130522115304308F499270E9439
:1031B000EA160E94A01117C081E0A0CF80959095DB
:1031C00082239323BECFC601905281159043A0F471
:1031D000C60199270E94EA168091BC039091BD0315
:1031E0008C159D0531F31093BB030093BA03CDB743
:1031F000DEB7E8E00C94A133C601ECCFA8E0B0E064
:10320000E4E0F9E10C947B337C01DC0114968C91B1
:10321000882309F464C161E0C7010E94260D8C0176
:10322000F7018581882331F18091B4049091B50430
:10323000009701F108171907E9F0FC01FF27887FC3
:103240009927892B09F069C0A4E0EE0FFF1FAA950A
:10325000E1F7E25BFD4F8581846085831183008304
:10326000CF010E9479111092240561E0C7010E94EC
:10327000260D8C01D70115968C91882309F4BBC0CB
:10328000C80197578038910508F0E8C0D02EBFE0FC
:10329000B01708F415C18FEF93E00E941D3481111F
:1032A0000FC10CE613E0D1103BC0F4E04F2E9E019D
:1032B0002F5F3F4F390133243A94D301E42D1D92FF
:1032C000EA95E9F76801FFEFCF1ADF0AC8010E940B
:1032D0001D348983882309F4F3C08130D1F4580167
:1032E00022E0A20EB11CC6010E941D34582E8A8312
:1032F000882309F4E5C08FEF850D8330F8F4680169
:1033000033E0C30ED11CC5010E941D348B8388237A
:10331000F1F1C3010E9477173AC0F0E0E0E09BCFE3
:103320000115E4E01E0709F4CBC0C8010E941D345A
:10333000811101C0DA940F5F1F4FB5CF8BEF850D60
:10334000833068F5480143E0840E911CC5010E945A
:103350001D348B8364018823D1F0680154E0C50ECD
:10336000D11CC4010E941D348C83882381F08B8181
:103370009C818130AFEF9A0710F0982F8827B6E034
:103380005B1639F0E7E05E1639F00E9424278601CB
:1033900094CF0E94FF26FBCF0E948626F8CFF4E050
:1033A00065015F12F4CFC5010E941D34B82E68017B
:1033B00024E0C20ED11CC80103960E941D34BB201C
:1033C00009F47EC0882309F47BC0482F4150550B77
:1033D000349EC001359E900D1124AB2DA150BB0B26
:1033E0008A0F9B1F019798F2EFE9FFE03197F1F701
:1033F00000C00000F7CF680127E5D21A3FEFC316DF
:10340000D10409F058F564E472E08C2D0E94780D27
:10341000892B21F5C60174E0880F991F7A95E1F791
:10342000FC01E25BFD4F22812130A1F52091440295
:1034300030914502232B91F02091460230914702B2
:10344000232B61F0209148023091490240914A02B9
:1034500050914B02242B352B232B21F1D7011596AC
:103460005C90552009F43FC00E35BCE71B0729F1DD
:103470000F35ECE71E0741F00D35FCE71F0799F506
:10348000809100018823C9F01092000180E00E9421
:10349000841616C0223011F720914802309149025B
:1034A000232BE1F2FC01ED5AFD4F20812E7F20837A
:1034B000825B9D4F0E947911D1CF81E08093000102
:1034C0008091D101877059F0F7018581882339F007
:1034D0008091980382FF03C082E00E94020A28962E
:1034E000E2E10C94973380910001882309F4B9C478
:1034F000380120EE621A71084090DC018091CE0103
:10350000482A80919903482A38E06316710408F02C
:1035100087C098012770332781E090E001C0880FB1
:103520002A95EAF7552009F478C0482AD7018D91E9
:103530009C910E94670921E030E0190102C0220C31
:10354000331C8A95E2F7E0918104F0918204FE83B6
:10355000ED832091A6013091A70138872F836FE179
:10356000C62E63E0D62EB12CA12CB8E0AB16B10468
:1035700009F4D8C4411005C0D60112968C9181116E
:103580008BC0F601838190E082219321892B09F47D
:1035900083C08085982F977009F487E0F8E06F1654
:1035A000710408F057C0552009F450C08695817009
:1035B000882309F471C0D6018D909C9008151905D7
:1035C00019F4552009F468C0ED81FE81EC15FD0564
:1035D00009F462C0D6011D96ED91FC91309721F05F
:1035E0008081882309F458C0642DC6010E949C067E
:1035F000882309F451C00815190509F038C50115CB
:10360000110509F439C5511039C5EF81F8858E16B9
:103610009F0609F041C0512C31C58095482286CFC4
:10362000552009F468C41093A7010093A6010E94D5
:10363000DE04609378047093790480937A04909305
:103640007B041092800410927F0470CF82FB882745
:1036500080F9AECF552001F18170AACF0E9451169A
:1036600032C50497813A910558F46C2D8EE991E0AA
:103670000E940305552009F4F4C30E940F1120CFC6
:103680000E940F118FE39CE90197F1F700C0000041
:103690008C2D0E940217EECF9FEFA91AB90AAFE056
:1036A000CA0ED11C62CFDC012D913C910217130789
:1036B00009F0D1C35110D1C310927E0480E00E9462
:1036C0008416CFC3902F812F11C4F90144855585ED
:1036D00066857785C9010E947805D60115968C917B
:1036E00081FF34C4C6010E9460118091B40490919E
:1036F000B5040817190709F029C41092B5041092EF
:10370000B40424C490913601892F8E7F90FF81608C
:10371000809336010E94A01144C4809136018E7FAF
:10372000F7CF809136018F7E013E110531F0053EC5
:103730001105E9F4809136018F7D809336018091E7
:10374000360180FF19C0D70115968C9108321105FA
:1037500020F50E31110508F071C00430110578F51F
:10376000882351F01092BD031092BC0305C0C8011C
:1037700090528115904318F7F70185810737FCE7D0
:103780001F0709F4D0C008372CE7120709F013C44B
:10379000882309F4D7C082E0C9C00933110558F461
:1037A0000D32110518F40B321105D1F690919F04DA
:1037B00092FDD6CF08C004361105C1F3D1CF909148
:1037C0009F0494FDCDCF882309F4A6C08091DC012D
:1037D00090919903892B8D7FB1F11092BD031092C6
:1037E000BC0380919F0481FD2EC0F80143E0F69553
:1037F000E7954A95E1F7EE71FF27E656FC4F9801F1
:103800002F70332781E090E002C0880F991F2A951E
:10381000E2F78095909520813181822393239183D3
:10382000808360E0C8010E943F188091DC018D7F99
:103830000E94F50882E00E94020A42CE90919F0405
:1038400093FD8ECFC0CF89E0F701A0E2B2E00190F6
:103850000D928A95E1F71092230210922202809134
:10386000BC039091BD0308171907D1F520919F045F
:1038700025FF36C03091360131FF02C026FF30C02F
:103880002091BA033091BB035601A21AB30AB701C3
:103890000E948C0DA816B90618F58091990381FF36
:1038A00008C08091360180618093360182E00E94D9
:1038B00025098091990385FF08C0809136018062B7
:1038C0008093360180E20E94250960913601669559
:1038D00061708091BC039091BD030E943F18F0CDB0
:1038E0008091DC0190919903982B2091360191FBF6
:1038F00021F9209336018D7F0E94F5081093BD03B6
:103900000093BC03D092BB03C092BA0380913601EE
:103910008460809336018ECF970140E0B601C801E4
:103920000E944F18CDCD882349F081E00E94190AEA
:1039300043E062E081E00E94D509C2CD81E00E94AF
:10394000F509F6CF82E0FBCF0B353CE7130749F1D1
:103950000C354CE71407D9F00A351C4709F040C371
:1039600081E01CC00E94BF118FEF94E3ACE0815056
:103970009040A040E1F700C000000E94BE046FEF3D
:103980007FEF90E080E00E9459340E941C168091E5
:10399000980382FB882780F991E089270E94AA0D6D
:1039A0001FC380E0FBCFF70185810081118188234F
:1039B00069F0C8010E94B10CD82E682FC8010E947E
:1039C0009B09B8018D2D0E94940C11C3C8010E945F
:1039D0006709D82EF6CFE02FEF70DE2E802F807F84
:1039E00019F0D29490EFD922CC20A9F0DD2059F023
:1039F00080E2810F883010F0111107C08D2D0E94D8
:103A00002C090E940F11812F3FC080912405D82AD4
:103A1000D0922405F6CF812F0E945116DD20B1F1FE
:103A200080E2810F883010F0111104C08D2D0E94AA
:103A3000250903C08D2D0E941E090E940F1126C06A
:103A4000F02FFF70DF2E802F807F803219F0D2940C
:103A500080EFD822112351F0113009F499C0CC2005
:103A600009F4A5C0BB2009F449C0CDCF80919803CB
:103A700082FD40C0CC20C1F1DD2029F08D2D0E94B7
:103A80002C090E940F1180E00E940217A92DA85056
:103A9000BB0B149710F40E946705812F902F0E9492
:103AA0003F0A8111B8C11092A9011092A801AA2061
:103AB000B1F08091D10180FD12C0D70115961C9202
:103AC0008695869586950E94190AC7010E94FE1860
:103AD0008091D1018695869586950E94F50960E0D2
:103AE000C7010E94260DFBCC80E00E945116DD200C
:103AF00069F29CCFCC2091F1B11004C08D2D0E94B1
:103B00004A16C4CF21E0B21211C08090DC018D2D85
:103B10008821D81609F4BACF0E94EA049093DB01F9
:103B20008093DA01D828D092DC01B0CF8091A00434
:103B3000823008F4ABCFB812A9CF8D2D0E944A165F
:103B40008D2D0E9409098091CE019D2D9823D916B3
:103B500009F49CCFD82AD092CE0198CFB1100AC0D8
:103B60008D2D0E9443168D2D0E9409098D2D0E94D6
:103B700053098CCF8091A004823008F487CF31E0C4
:103B8000B31284CF809199038D2109F47FCFE8CFC0
:103B90008091A604CC2021F08B1508F477CFAECF0E
:103BA000B81608F073CF8D2D0E9443166FCFBB203F
:103BB000D1F38091A4049091A504193321F0809150
:103BC000A2049091A3040E94C00B812F0E94511661
:103BD0005DCF802F86958695837069F0813009F0DE
:103BE00055CF812F902F9370C11002C080E090E0DC
:103BF0000E941D054BCF812F902F9370C11002C0E2
:103C000080E090E00E94420541CF6C2D812F0E9400
:103C10005A0A3CCF802F837091F5C11037CF412FC6
:103C2000429546954770440F440F812F8F70042EA4
:103C300001C0880F0A94EAF7212F207114FF07C0F2
:103C40002FE030E001C0220F4A95EAF72095302F8F
:103C5000369536953370323069F050F44091110248
:103C6000313029F0822B84230E943C0A0FCF842B11
:103C7000822BFACF282B809111028227F5CF8695CF
:103C8000CC2011F0802F8170882309F4FFCE412FC2
:103C9000429546954770440F440F812F8F70042E34
:103CA00001C0880F0A94EAF7212F207114FF07C082
:103CB0002FE030E001C0220F4A95EAF72095302F1F
:103CC000369536953370323069F050F440911202D7
:103CD000313029F0822B84230E94D209D7CE842B45
:103CE000822BFACF282B809112028227F5CF402F0A
:103CF0004F70D42ECC2029F0842F0E94190A812FD6
:103D0000FECE812F0E9443168D2D0E94F509BECE56
:103D1000123F89F160F4103FB9F0113F81F0CC20DF
:103D200009F474C0B1106FCE802F8F7128C0133F7B
:103D300049F1143FA1F78091980382FD2FC0802F95
:103D40008F71CC2011F31BC08091A604CC2079F098
:103D5000B81608F09BCE202F2F7181E090E001C0B3
:103D6000880F2A95EAF7909112028927B5CF8B1513
:103D700008F48CCEF0CF802F8F71C110C6CF0E9477
:103D8000190A84CE80E0CC2009F4A6CF81E0902FE0
:103D90009F7101C0880F9A95EAF79ECF8091A00489
:103DA000823008F1CC20A9F09091D1019770943025
:103DB00041F40E943209802F8F710E94F509A12CD5
:103DC00065CE63E0B816D8F7802F8F710E94250A60
:103DD000F6CFB81620F00E94320964E0F5CF81E0FA
:103DE0000E94020AECCFCC2031F063E0802F8F716B
:103DF0000E94250A4BCE81E00E94020A51E05B1529
:103E000008F044CE82E00E94020A40CEB110D1CE2A
:103E1000802F8F717ACFCC2019F0B11044CE47CECD
:103E2000B11041CE20E0F701408151816281738160
:103E3000848195810E94010D8091A10483FF33CE7E
:103E40008091A8019091A901029709F02CCE812FB1
:103E50000E946A1728CE552021F0FC01808585FF3D
:103E60002DCCC80197558F3F910511F008F06EC019
:103E7000C801887F9927892B09F022CBF801FF27F9
:103E800054E0EE0FFF1F5A95E1F79F01225B3D4F73
:103E90006901D70115968C91ED5AFD4F908180FBF9
:103EA00090F99083882309F410CC0E94EA0490933F
:103EB0001F0280931E02F60182818F5F82838091B0
:103EC000240590919903892B83838091DC0184835D
:103ED0004681578166857785C6010E947805D6019F
:103EE00015968C9181FFEECB90E080E09093B40426
:103EF0008093B5042BC08091A6019091A70108176B
:103F0000190781F41092A7011092A601109278046B
:103F10001092790410927A0410927B04109280041B
:103F200010927F048091810490918204009709F49B
:103F300098CFE8E06E16710408F0B5CB642D0E94AE
:103F40009C06811103C081E00E94841680919F0429
:103F500080FF12CC0E94EA046C01F701858188235E
:103F600009F4DFCB8091360182FF08C020E232E005
:103F700040E0B60190E080E00E944F180431FCE779
:103F80001F0709F4CACB05312CE7120709F4BACB95
:103F900003313CE7130729F4809136018160809357
:103FA0003601C80190528115904308F0C8CB109299
:103FB000BD031092BC03D70115968C91882381F024
:103FC0000330BCE71B0709F4DACC08F0BDCC0115BF
:103FD000FCE71F0709F4C6CC01301C4709F4D5CC17
:103FE000D70117968D919C91009709F4DCCC0E9423
:103FF000FB07182F092FD7011596CC901597169609
:10400000BC90B2943FE0B3228091D101877001F15E
:10401000AC2CCC20F1F0892F807F803461F080E2DD
:10402000810F8830A8F0892F807E803221F41230F1
:1040300078F0BB2069F08091980382FF09C082E08C
:104040000E94020A8091D1018770AA24A394811151
:10405000A12C902E92942FE09222BBE0B91508F487
:1040600015CDE92DF0E0ED57FB4C0C94DA338114BB
:10407000910409F0CACA512C912C812C80E00E9435
:104080008416D0928204C092810481E080937E04E1
:104090008FE08A9DF0018B9DF00D1124E15EFC4FB5
:1040A000858180937C0451100EC08114910459F0D5
:1040B000808191819C0124503109213A310508F019
:1040C000CDCA0E94F6048FE08A9DF0018B9DF00D11
:1040D0001124E15EFC4FC680D780C6019A958115F8
:1040E0009F4110F420EED22299249394C6010197A7
:1040F0008F339E4708F0912C8FE08A9DD0018B9DD5
:10410000B00D1124A15EBC4F1996ED91FC911A9748
:10411000309731F01B966D917C9181E00995982242
:104120009920B1F08FE08A9DF0018B9DF00D112454
:10413000E15EFC4F868197810E94320B80937D0463
:10414000C60148E06416710408F08BCA0E944B0651
:104150000E940F118FCAB0E0A0E0E1EBF0E20C94F6
:1041600086338091CB01807F09F054C08091CA01D1
:10417000882309F44FC0E091230589E0D82E80916F
:10418000DA048E1709F446C00E2F10E0ED9DF00101
:104190001124E552FB4F8481882309F440C0D09E4E
:1041A000E001D19ED00D1124FE01E552FB4F91811B
:1041B0008091C601981333C090818091C5019813F6
:1041C0002EC0858181112BC0E280F3808091C701D0
:1041D0009091C801E81AF90A60E085EC91E00E942C
:1041E000260D65EC71E00E948C0DE816F906B8F416
:1041F0008091CB018F7080618093CB01CF51DB4FD9
:1042000088818F708061888385EC91E00E94FE1820
:104210000E945D09CDB7DEB7E7E00C94A233F80148
:104220003196E770ACCFA8E1B0E0E9E1F1E20C949F
:104230007E338C0186E0F801DE01539601900D92E9
:104240008A95E1F7D80114967C9014971596EC9016
:1042500085ECA82E81E0B82E8091C90181112AC079
:10426000711003C0FF24F3941CC0EE20F9F0C801C4
:104270000E94ED0CF82E8823C9F089E0F801A5EC26
:10428000B1E001900D928A95E1F78091C9018130EA
:1042900031F48091C5019091C6010E94E00C0E940A
:1042A000AB208F2D6896EFE00C949A33C8010E94E2
:1042B000FE18D8CFF80150806180C280D38060E0C2
:1042C00085EC91E00E94260DF090CA018091C70113
:1042D0009091C8014601881A990A60E085EC91E046
:1042E000FF2009F428C10E94260D65EC71E00E94B0
:1042F0008C0D8816990608F0D1C0772009F4B2CF4A
:104300008091CB01382F307F2091C601D8011196C2
:104310009C911197311171C029131FC02091C501C3
:104320009C9129131AC04091CC015091CD01179650
:104330002D913C914217530781F4E11054C08F70C6
:1043400080618093CB0185EC91E00E94FE18809102
:10435000CB01F8018683F12CA4CFE11044C0662D77
:10436000852D0E942A03E82E882381F08091A104E4
:1043700080FFF1CF85EC91E00E94FE1889E0E5EC2A
:10438000F1E0DF011D928A95E9F7E5CF5B8A6C8A3F
:104390008B899C890E94E00C292F22952F70243054
:1043A00058F49F70223088F0992399F0F801968193
:1043B000907F79F4FE2C75CF2A5F2F70223068F041
:1043C000C8010E94FE18EF2CF5CF992311F0882325
:1043D00089F3805E883070F3F3CF803F58F3815FBC
:1043E000833070F7E7CF8091CB0181608093CB0160
:1043F0008091A10481FDAFCFBDCF291320C02091B2
:10440000C5019C9129131BC04091CC015091CD0155
:1044100017962D913C9118974217530781F4E1109C
:104420000EC016968C93C8010E94FE1889E0F80110
:10443000A5ECB1E001900D928A95E1F732CFC80169
:104440000E94ED0C882309F431CFEE2009F42ECF21
:104450008091CB018032B8F02091C5013091C60126
:104460003B872A87DD86CC869091C9019E871F866F
:10447000888B8091CC019091CD019A8B898BCE0154
:104480000A960E94FE1889E0F801A5ECB1E00190BF
:104490000D928A95E1F70E94AB20E4CE8091CB018A
:1044A000982F907F09F466CF772009F4DBCE209116
:1044B000C601F801918129131AC02091C50190818C
:1044C000291315C04091CC015091CD012781308531
:1044D0004217530761F4E1100AC08683C8010E94A5
:1044E000FE1889E0D5011D928A95E9F7DACEC80158
:1044F0000E94ED0C882309F4D9CEEE2009F4D6CE23
:104500008091CB01803208F4BECF2091C50130915B
:10451000C6013A832983DC82CB829091C9019D83B5
:104520001E828F838091CC019091CD0199878887DD
:10453000CE010196A6CF0E94260D65EC71E00E9487
:104540008C0D8816990608F055C0772009F48ACE9C
:10455000FE2CEE2009F4AACE9091C601F8018181CB
:1045600098133AC09091C5018081981335C020916D
:10457000CC013091CD01878190852817390761F5ED
:10458000A090C701B090C80160E085EC91E00E9466
:10459000260D8091A10482FD49CFCA18DB088091C5
:1045A0009C0490919D04C816D90608F03FCF8091D5
:1045B000CB0180FD3BCF982F907F09F437CFD801F6
:1045C00016968C931697903F09F42DCF982F907FD5
:1045D000905F8F70892B25CFC8010E94ED0C81114F
:1045E00052CF8091CB0181608093CB01C8010E94A2
:1045F000FE1857CE89E0F50111928A95E9F751CE60
:10460000A2E1B0E0E6E0F3E20C9489330A871B876D
:104610002C873D874E875F87688B798B8A8BCE018D
:104620000A960E94132181110CC089E0FE013A967E
:10463000DE01119601900D928A95E1F78E85811128
:104640000BC019E0809123059091DA04891331C0E1
:104650006296E4E00C94A5332091DA0430E0C901BD
:10466000019687709927409123054817190699F0FC
:1046700099E0929FD001939FB00D1124A552BB4F9A
:10468000FE01319601900D929A95E1F78093DA043C
:104690000E945D09D6CF0E94BF111092DA041092D9
:1046A000230589E0E5ECF1E0DF011D928A95E9F749
:1046B000C8CF819FC001112485529B4F0E941321B6
:1046C000882331F28091230590E001968770992725
:1046D00080932305B7CFEF92FF920F931F93CF9351
:1046E000DF938091F903882361F0E091C0038DE0AE
:1046F000F82E8091F903E81748F01092F903109210
:10470000C003CDB7DEB7E6E00C94A333EE24E39408
:10471000EE0EE092C003CE2FD0E0EF9DF001112409
:10472000E650FC4F84818823E9F087819085892BAE
:1047300021F481859285019659F4008111812281AD
:104740003381448155816681778180850E94002371
:10475000FC9EF001FD9EF00D1124E650FC4F1482EA
:1047600010922405EE2DC5CF10926D0410926C04AA
:104770001092370180916B0480936A040E94EA06CC
:104780000E946B230895B0E0A0E0E9ECF3E20C9402
:104790007C33C0916A0497E0992E01E010E02DE08F
:1047A000322E34E0432E5524539480916B048C13A5
:1047B00009C00E946B230E94EA06CDB7DEB7E1E193
:1047C0000C949833D0E0FE01EE0FFF1FEE59FB4F23
:1047D00080819181989ED001999EB00D1124AF5394
:1047E000BC4F14962C911497211159C06090F90375
:1047F000EAEFF3E030E020E0812C5D01261508F0BF
:104800004CC0E384F484D501CD90DC906FEF7FEF52
:10481000712C472D50E0DA01AA0FBB1FAC0DBD1D56
:104820000D90BC91A02D109731F0EA16FB0609F40B
:10483000BA017394EECF6F3F7607A9F1D80102C099
:10484000AA0FBB1F6A95E2F78A2AB801072C02C09B
:10485000660F771F0A94E2F7AB01415051098416A5
:10486000150601F5329EF001339EF00D1124E6503D
:10487000FC4F989ED001999EB00D1124AF53BC4FB0
:1048800012962D913C911397308727834482108292
:1048900011829287818715965C920E94BC062196B0
:1048A000C37083CF14822F5F3F4F3D96A7CFAEE1F9
:1048B000B0E0EDE5F4E20C947B334B8B5C8B6D8BBD
:1048C0007E8B8F8B988F882349F08091A8019091DF
:1048D000A90101969093A9018093A801888D811167
:1048E00010922405188A198A1A8A86E0FE017396A6
:1048F000DE011A9601900D928A95E1F78091980356
:1049000082FF1EC08091860490918704892BC1F09C
:104910000E94EA042091CF013091D001821B930BB9
:1049200020918604309187048217930720F08091AC
:10493000D10182FFE7C10E94390981110E94EA0872
:104940008E85882389F061E0CE010A960E94260DAB
:104950006C018F8520E5C2162CE7D20689F48823E6
:1049600029F181E0809337010A851B852C853D85DF
:104970004E855F85688979898A890E940023CDC028
:1049800031E5C3163CE7D30629F4882379F00E9469
:10499000B423EACF42E5C4164CE7D40639F48823A1
:1049A00029F0809137018111F2CFDBCF91ECE92E14
:1049B00093E0F92E412CB12CA12C88248394912CC6
:1049C000BE016F5F7F4F7A8F698F22242394F70196
:1049D0004081518166246A94762C20E0822F90E0F9
:1049E000FC01EE0FFF1FE40FF51F6081718161155F
:1049F000710531F0C616D70609F43C012F5FEECFE2
:104A0000312CFFEF6F167F0609F448C0F70144818F
:104A100030903701832D411180E0F82FF1703F2E47
:104A2000F701558086819F85992309F4F7C03320CB
:104A300009F4F4C000919A0410919B04511013C022
:104A4000A401062C01C0440F0A94EAF7842B868344
:104A50008091BE039091BF038017910720F41093BB
:104A6000BF030093BE03C40102C0880F991F2A959B
:104A7000E2F70197F70126812817190679F480914A
:104A80006C0490916D04009709F44BC00E94CF0410
:104A90000817190708F045C0F70124824328FFEFE3
:104AA000AF1ABF0A27E0E20EF11C38E0A316B104EA
:104AB00009F08DCF8F85882309F410C1442009F4B3
:104AC0000DC10E94EA0490936D0480936C04809160
:104AD000F903883010F591E0980F9093F90399E06D
:104AE000FE013A96DE01119601900D929A95E1F73A
:104AF0004DE0849FC001112486509C4F29E0FE01A7
:104B00003196DC0101900D922A95E1F72FEF3FEFEE
:104B1000FC0132872187D486C3866E96E2E10C942D
:104B2000973380916A0450916B04982FF0E0E0E095
:104B3000851314C090936A04EE16FF0609F4AECFF5
:104B400090E0FC01EE0FFF1FEE59FB4FB182A082F7
:104B500001968370992780936B04A0CF682E712CE7
:104B6000F301EE0FFF1FEE59FB4F20813181F7E07B
:104B7000F29FD001F39FB00D1124AF53BC4F2D9184
:104B80003C9111973E8F2D8F40E020E030E0E32FE5
:104B9000F0E0EE0FFF1F6D8D7E8DE60FF71F008199
:104BA000118101151105E1F0F7010190F081E02D6F
:104BB000FC8FEB8F20E005C00617170709F4432D83
:104BC0002F5FE22FF0E0EE0FFF1F6B8D7C8DE60F65
:104BD000F71F608171816115710571F73F5FD7CF54
:104BE0004423C9F0F701231708F0FD012482EE16D3
:104BF000FF0621F490936A04342E50CF891305C028
:104C0000AE17BF0711F49F5F937093012F5F3F4F63
:104C1000822F83708DCFF0E0E0E0F7CF90E051106D
:104C200020C0B40102C0660F771F2A95E2F79B01EE
:104C3000215031092817390731F4442309F44CC0B5
:104C4000C5010E94BC06C401062C01C0880F0A944D
:104C5000EAF7982F9095F701868189238683352C72
:104C60001DCFAC01062C02C0559547950A94E2F77A
:104C7000BA01617077279C01215031098223932367
:104C8000892B31F5672B21F1F70182819381892BE3
:104C9000E1F0E98DFA8D27E011922A95E9F70E945B
:104CA000EA04282F8B839C8334E03D83F7018281C3
:104CB0009381782F8887998709811A813C8144E004
:104CC0005E816F81892F0E940023F7011582BBCF7F
:104CD000F42FF1705F2EB7CF532CB5CF90916A04AB
:104CE00080916B04981729F00E94C323411015CFBF
:104CF0003BCE0E946B2310926D0410926C040E94B4
:104D0000EA06F4CF82E00E94020A15CEA6E0B0E0E7
:104D1000ECE8F6E20C948B3390933B0280933A02DA
:104D2000811520E2920730F40E94EA162696E2E00E
:104D30000C94A73380EF89838A830E94EA04816000
:104D4000682F9C838B8349815A817C8181E090E02C
:104D50000E945724EBCF0F931F93CF93DF938C01C7
:104D6000EB0164E472E08C2F0E94780D892BA1F492
:104D70008091A2049091A3040E94C00BDD27C45C23
:104D8000DD4F8881F801128218828330F1F048F4F7
:104D9000813059F0823081F0DF91CF911F910F91D6
:104DA00008958430B9F08530B9F78091440290912C
:104DB0004502009789F306C0809146029091470210
:104DC000009799F30E948626E7CF80914802909140
:104DD0004902F6CF80914A0290914B02009791F7D9
:104DE0002091440230914502809146029091470201
:104DF00021153105F1F2009729F7C901E3CFA6E0AB
:104E0000B0E0E5E0F7E20C948B3390933B028093A3
:104E10003A02811520E2920730F40E942718269664
:104E2000E2E00C94A73380EF89838A830E94EA042E
:104E30008160682F9C838B8349815A817C8181E0CA
:104E400091E00E945724EBCFCF93DF93EC010E94B7
:104E5000FF268091A2049091A3040E94C00BCE0172
:104E60000E948626DF91CF9108950F931F93CF93D1
:104E7000DF938C01862F64E472E00E94780D892B09
:104E8000B1F4C0914402D0914502209781F0F8011D
:104E90008281833051F4CE010E942427CE010E94EA
:104EA0002427CE010E94242702C08430D0F7DF914E
:104EB000CF911F910F9108950F931F93CF93DF937D
:104EC0008C01EB0164E472E08C2F0E94780D892B39
:104ED00009F05CC0FE01FF27D80112968C91129751
:104EE000E45CFD4F8130B9F415969C9192FF02C0AD
:104EF00080830AC090FFFCCF82E0808380914602CD
:104F0000909147020097B9F4809144029091450234
:104F10000097E1F110C08230B9F515968C9182FDB1
:104F200028C080FD0BC083E080838091480290916F
:104F30004902009701F10E94FF2628C084E0808387
:104F400080914A0290914B020097A9F78091440208
:104F5000909145020097F9F00E9424278091460223
:104F600090914702009739F7809144029091450251
:104F7000E2CF85E0808380914402909145020097C2
:104F800029F00E942427F0CF86E08083DF91CF9123
:104F90001F910F9108958091460290914702B8CFDA
:104FA000A6E0B0E0E6EDF7E20C9489330E94EA0453
:104FB0008C018091DD019091DE018017910781F0D5
:104FC00019821A820E94EA04682F49815A81792F36
:104FD00080E090E00E9457241093DE010093DD01F1
:104FE0002696E4E00C94A5331F920F920FB60F9211
:104FF00011242F933F934F935F936F937F938F93DE
:105000009F93AF93BF93CF93DF93EF93FF93D09191
:10501000E900DF708091EC00C82FC17080FDC0E80E
:105020001092E9008091F000877F8093F0007894DF
:105030000E94E6111092E9008091F0008860809350
:10504000F000CD2BCF70C093E900FF91EF91DF917D
:10505000CF91BF91AF919F918F917F916F915F9110
:105060004F913F912F910F900FBE0F901F90189569
:105070001F920F920FB60F9211242F933F934F93CD
:105080005F936F937F938F939F93AF93BF93EF93B0
:10509000FF938091E10082FF09C08091E20082FFCE
:1050A00005C08091E1008B7F8093E1008091DA0060
:1050B00080FF24C08091D80080FF20C08091DA005A
:1050C0008E7F8093DA008091D90080FF9DC080E1BF
:1050D00089BD82E189BD09B400FEFDCF81E08093E6
:1050E000D0048091C304811109C00E9460030E9412
:1050F00001048091E20084608093E2008091E100ED
:1051000080FF17C08091E20080FF13C08091E20011
:105110008E7F8093E2008091E20080618093E200C4
:105120008091D80080628093D80019BC85E080937C
:10513000D0048091E10084FF2BC08091E20084FFC5
:1051400027C080E189BD82E189BD89B5982F917022
:1051500080FFFBCF8091D8008F7D8093D800809115
:10516000E1008F7E8093E1008091E2008F7E80934A
:10517000E2008091E20081608093E2008091D1049E
:10518000882309F447C084E08093D0048091D00440
:105190008091E10083FF27C08091E20083FF23C05C
:1051A0008091E100877F8093E10082E08093D004CA
:1051B0001092D1048091E1008E7F8093E100809174
:1051C000E2008E7F8093E2008091E2008061809314
:1051D000E20042E060E080E00E94CF038091F000B6
:1051E00088608093F000FF91EF91BF91AF919F9104
:1051F0008F917F916F915F914F913F912F910F9080
:105200000FBE0F901F90189519BC1092D0041092E9
:10521000C30474CF8091E30087FD93E09093D004A2
:10522000B5CF78941F921FB61F9211248F939F932E
:10523000AF93BF938091BF049091C004A091C1042B
:10524000B091C2040196A11DB11D8093BF0490933B
:10525000C004A093C104B093C204BF91AF919F91C9
:105260008F911F901FBE1F9018951F921FB61F92FF
:1052700011248F939F93AF93BF938091BE048111AC
:1052800013C08091BF049091C004A091C104B0915B
:10529000C2044196A11DB11D8093BF049093C00428
:1052A000A093C104B093C204BF91AF919F918F911D
:1052B0001F901FBE1F901895CDB7DEB7C054D109FF
:1052C0000FB6F894DEBF0FBECDBF85B7806885BF2F
:1052D00085B7806885BF84B7877F84BF0FB6F89491
:1052E000A8958091600088618093600010926000B2
:1052F0000FBE80E890E00FB6F89480936100909321
:1053000061000FBE88EC97E090939D0180939C0113
:105310000E94A3070E94760E0E94F20D0E94520D79
:105320000E9460030E9401048091E20084608093E7
:10533000E20078948091D0048823A1F01091E900D4
:105340001F709091EC00892F817090FD80E8182BE0
:105350001092E9008091E80083FD0E94E6111F7021
:105360001093E90082E084BD93E095BD9AEF97BD6C
:1053700080936E00109201021092020210920302BA
:10538000109204020E944C0C811102C00E949115DF
:105390008091D80080618093D8002AE12A95F1F7A6
:1053A00000C08091D900182F117080FD04C00E94A8
:1053B00060031092D0041093B6041093B7041093B6
:1053C000250111110E9419328091250181112CC0F3
:1053D00085E0EDE3F1E0DE01919601900D928A9572
:1053E000E1F789A1809320018AA1809321018BA1FB
:1053F000809322018CA1809323018DA180932401AD
:1054000087E0E2E4F1E0DE01119601900D928A95C9
:10541000E1F7FE013196A9E1B1E0CE0108962191B4
:105420002D93E817F907D9F78091250195E08111AF
:1054300090E09093100285E0891B80930F0200E2B8
:1054400011E045E2E42E41E0F42ED8018D918D016A
:105450008F3F11F00E94CA07E016F106B1F709E18B
:1054600011E030E2E32E31E0F32EF80181918F015B
:105470008F3F11F00E94CA07E016F106B1F78AE0EB
:10548000EEE2F2E0DF01282F1D922A95E9F7E5E030
:10549000F2E0DF011D928A95E9F790E080E00E943A
:1054A0002534853E9E4F21F40E944C0C811163C02F
:1054B00065EE7EEF90E080E00E94593460E082E08B
:1054C00090E00E943B3481E08093110261E083E030
:1054D00090E00E943B3460E074E184E090E00E9440
:1054E000593460E086E090E00E943B3460E087E061
:1054F00090E00E943B3440E050E0BA0188E090E048
:105500000E944D3460E083E290E00E943B3460E012
:105510008CE090E00E943B3460E08DE090E00E94DF
:105520003B3419821A821B821C821D821E821F82BA
:10553000188648E050E067E170E0CE0101960E94D5
:105540002B3440E050E0BA018FE190E00E944D34EE
:1055500080E00E94FD0B0E94911540E050E0BA01EE
:105560008FE090E00E944D3440E050E0BA0183E1CA
:1055700090E00E944D3482E090E00E941D348093C0
:10558000130284E090E00E94253490939803809366
:1055900097030E94AF0FEFEFF6E721E0E150F040F4
:1055A0002040E1F700C000000E94AF0F80912E0262
:1055B00080FF08C06FEF7FEF90E080E00E945934D9
:1055C0000E94BE0483E090E00E941D340E943C0AC9
:1055D0008091B604811102C00E941C3286E291E0E3
:1055E0009093BB048093BA048EE292E03AE0380FC5
:1055F00021963FAF21973324339422242394CE0164
:105600008B969BAF8AAF8E010F5F1F4FDE01139603
:10561000BDAFACAF8091D004853079F480E4F82E32
:1056200090E1E92E22E1D22E8091D004853009F458
:1056300055C00E94BF110E9467050E94AF0FA4E1F0
:10564000EA2EA2E0FA2EBEE2AB2EB2E0BB2E2EE195
:1056500032E0D501F70191918D912E173F0709F4A2
:1056600071C09817C1F34090B604FEE2CF2EF2E06D
:10567000DF2E912CD6018D906D01F70151907F01A5
:10568000581429F1712C662463945824852D8621A1
:10569000B1F04420A1F07CAA9DAA0E94EA049FAB2D
:1056A0008EAB28AE91E0862D882109F490E099AF69
:1056B0004CA95DA96EA97FA988AD0E945724739457
:1056C000660CF7E07F12E2CFF70131978082939466
:1056D0002AE09212CFCF0E94E10738C08091D00417
:1056E000843019F11092BE04E8E1F0E00FB6F894AE
:1056F000A895E09360000FBEF092600083B7817FB1
:10570000846083BF83B7816083BF7894889583B7B3
:105710008E7F83BF0FB6F894A89580916000886152
:1057200080936000109260000FBE0E94AF0FEEE207
:10573000F2E081918111CDC521962FAD21972E13D5
:10574000F8CF72CF98138FCF0E94D0278091B604E4
:10575000882309F4BFC080917F0490918004892B35
:1057600009F43EC040917404509175046091760430
:10577000709177042FB7F8948091BF049091C00482
:10578000A091C104B091C2042FBF841B950BA60B3E
:10579000B70B409170045091710460917204709144
:1057A000730484179507A607B707D0F080917F048C
:1057B000909180040E9427181092800410927F0418
:1057C000109274041092750410927604109277046B
:1057D000109270041092710410927204109273046B
:1057E000C090B404D090B504C114D10469F1809183
:1057F0001E0290911F020E94CF047C0189E0AAAD95
:10580000BBAD1D928A95E9F7BE01655D7F4FC6016C
:105810000E948C0D8E159F05B8F42091B404309130
:10582000B504C9019927287F3327232B09F004C128
:10583000E4E0880F991FEA95E1F7825B9D4FFC0138
:10584000258122FF0E94791180913701882301F17F
:1058500080916C0490916D040097D1F00E94CF0468
:105860002091BE033091BF032817390788F4909127
:105870006A0480916B04981709F4E1C00E94C32365
:105880001092BF031092BE0310926D0410926C042C
:1058900080919F0480FF1EC08091360182FF1AC054
:1058A0000E94EA042091BA033091BB03AC01421B71
:1058B000530B20913401309135014217530750F0BA
:1058C00020E232E041E0BC018091BC039091BD0335
:1058D0000E944F1886E0EEEAF4E0D80101900D92A4
:1058E0008A95E1F78090AF04D090B004E090B104C5
:1058F000C090B204F090B3041092B0041092B104BE
:105900001092B2041092B3048D2D8E2991F08091E3
:10591000AC049091AD040E94CF04AC01909183043B
:10592000992309F495C0809132018417150608F473
:105930009DC08F2D8C2991F08091AA049091AB0489
:105940000E94CF04AC019091A804992309F4C8C027
:10595000809130018417150608F4D0C08091AF04FF
:10596000881117C08091B004882311F08D1111C0E7
:105970002091B104222311F02E110BC09091B30499
:10598000992311F09F1105C03091B204332309F41B
:10599000E9C40E947E0586E0F801AEEAB4E0019019
:1059A0000D928A95E1F70E94670590912902891767
:1059B00021F0809329020E94DE048091D00484307B
:1059C00009F028CE83E08093E9008091E80082FF0F
:1059D00021CE8091E80090E085FF0AC00E947F03FD
:1059E00070E2C72ED12C7801882309F4CBC091E056
:1059F0008091E8008B778093E800992309F40ACE20
:105A0000E0903802F09039028981E114F10409F440
:105A1000C7C08E3F09F04AC18A81833020F085508B
:105A2000833008F043C1EA81EE3008F03FC1F0E076
:105A3000E157FB4C0C94DA3390E080E000CF0E94F9
:105A40006B2310926D0410926C040E94EA0620CF22
:105A500020913301FAE02F9F90011124241735077C
:105A600008F067CF9F5F9093830402C09F3FD1F7F8
:105A7000DD2059F00E94DE059FEF1D140CF491E02B
:105A8000899F802D11248093B004EE2059F00E944C
:105A9000DE0591E01E140CF09FEF899F802D1124EC
:105AA0008093B1048091B004882309F442CF909090
:105AB000B104992009F43DCF0E943D06882351F09E
:105AC0008093B004892D0E943D06882331F0809395
:105AD000B1042FCF3092B004F5CF3092B10429CF6A
:105AE000209131018AE0289F900111242417350765
:105AF00008F034CF9F5F9093A80402C09F3FD1F776
:105B0000CC2059F00E94A5059FEF1C140CF491E0E5
:105B1000899F802D11248093B204FF2059F00E94A8
:105B2000A50591E01F140CF09FEF899F802D112493
:105B30008093B3048091B204882309F40FCFC090FE
:105B4000B304CC2009F40ACF0E943D06882351F00B
:105B50008093B2048C2D0E943D06882331F08093FF
:105B6000B304FCCE3092B204F5CF3092B304F6CE3B
:105B70008091F100D7018D937D01B1E0CB1AD1085E
:105B800009F435CF8091E80085FDF2CF8091E800DF
:105B90008B778093E8000E947F03882399F327CFB7
:105BA0008C3009F4C4C060F5843009F4A7C050F407
:105BB000823009F46AC008F092C0813009F461C0F3
:105BC0008FEFB1C3863009F4AFC008F4A2C08B30A8
:105BD000B9F780916E0490916F04892B09F466C027
:105BE00040E250E0B80182E00E94630B3FEF41EEDB
:105BF00084E0315040408040E1F700C00000E0CC3C
:105C0000803109F4C3C088F58E3009F496C008F4D9
:105C100091C080916E0490916F04892B09F446C065
:105C2000EC80F12C3DE1E316F10408F03FC0CA809E
:105C3000DB80DC24CD24DC245801E00EF11EC601FB
:105C400084599C4FEA14FB0489F144E9C416D10439
:105C500028F4D50114966C910E943B34BFEFAB1A27
:105C6000BB0AEFEFCE1ADE0AEACF823109F493C005
:105C700008F48FC0833109F4B7C08E3F09F0A0CF7C
:105C8000D2CE1A8289E08B8311C08A81823009F4D6
:105C90006EC3833091F0813009F092CF0E94DE0410
:105CA0000E94E0336B837C838D839E8340E250E0CF
:105CB000B80182E00E94630BADCC80916E0490919C
:105CC0006F04892B99F3FE01339688E392E0D501A6
:105CD0002D915D0121938A179B07C9F7E7CF8A8130
:105CE000823009F06DCF6B817C818D819E810E9415
:105CF000E03387E290E00E943B34D8CF4C816B8147
:105D00008A810E94650C9827892798279E838D8316
:105D1000CDCF2D813E813227232732274C816B81C5
:105D20008A810E94260CC2CF0E940115BFCF80E15C
:105D30008A83BCCF1A8284E9A6CFEC80F12CBDE126
:105D4000EB16F10408F0B2CFCA80DB80DC24CD244E
:105D5000DC245801E00EF11EC60184599C4FEA1460
:105D6000FB0409F4A3CFE4E9CE16D10460F40E9449
:105D70001D34D50114968C93FFEFCF1ADF0A2FEF55
:105D8000A21AB20AE9CFF5011482F6CF0E94160CCE
:105D90008DCF84E0CDCFEC80F12CFDE1EF16F10446
:105DA00008F084CFCA80DB80DC24CD24DC245801B9
:105DB000E00EF11EC6018896AE14BF0409F476CF3A
:105DC00020E3C21622E0D20660F40E941D34D50101
:105DD00014968C93FFEFCF1ADF0A2FEFA21AB20AA4
:105DE000E9CFF5011482F6CFCC80D12C3DE1C3166A
:105DF000D10408F05BCFEA80FB80FE24EF24FE2470
:105E000040E3E41642E0F40608F050CF80E392E06D
:105E10008E199F098C159D0508F448CF370188E23B
:105E2000680E711C80916E0490916F0427014C0CD8
:105E30005D1C892BB9F5570191E0A922BB24E0FE36
:105E40000DC0C70187960E941D349D818927982720
:105E5000892781159C4711F48FEF8D83460140FE01
:105E60001AC0B1E08B1A9108E5E0F0E0EC0FFD1FDD
:105E7000E80DF91DFFAFEEAFC3018C0D9D1D0E9413
:105E80001D34AEADBFAD9C9181159C4721F48FEFC1
:105E9000EEADFFAD8083F801EA0DFB1D2FEFA814D6
:105EA000B90410F068011BC09481858181159C475D
:105EB00011F42483258342E0A40EB11C3296EFCF67
:105EC000A0E3EA16A2E0FA0620F4F60164810E943B
:105ED0003B34FFEFCF1ADF0A2FEFE21AF20AC701B5
:105EE00088964E145F0461F7E1CE88E0E9E4F1E0C2
:105EF000DE01919601900D928A95E1F780E2D8013A
:105F00001D928A95E9F786E0898388E0FE01B196C3
:105F1000DE01159601900D928A95E1F7C7CE88E9CA
:105F200089833A821B821C82C1CE8C81682F70E0EB
:105F3000762F66278B81860F972F911D092E000CD7
:105F4000AA0BBB0B65E0880F991FAA1FBB1F6A95A0
:105F5000D1F7AC01BD01405E5F4F6F4F7F4F4817D7
:105F600059076A077B0708F4A1CE8839E1E09E074C
:105F7000A105B10508F09ACE4939F1E05F07610546
:105F8000710520F048E951E060E070E0481B590BD2
:105F9000BC0163577E4FC8010E94E73387CE4AE1B8
:105FA00050E06FEF70E0CE0107960E9406348091BA
:105FB0006E048983EA821B821C8285E08D838E8336
:105FC00075CE81E090E0909339028093380282E3AD
:105FD00090E090932D0280932C020E94EA0490930B
:105FE0002B0280932A0262CEEF2861F1F0902E02FC
:105FF000E090330280912A0290912B020E94CF04FC
:106000008536910540F1E5FE26C0F0FE24C00E94D1
:10601000EA0490932B0280932A0280912C029091A3
:106020002D02019790932D0280932C02892B51F41D
:10603000109239021092380281E090E090936F0440
:1060400080936E0480916E048983809138028A83E4
:1060500080912C0218CE82E390E090932D028093E1
:106060002C02F0CF10926F0410926E041FCEEB80C2
:10607000FC8040E250E06FEF70E0C8010E940634FF
:1060800025E233E0A1E2B4E090E080E0AC014E5FB5
:106090005F4F4132510508F009CEF90165917491C5
:1060A000E616F70630F4800F911FFC0171836083C0
:1060B000CA01245F3F4FA217B30741F7F7CD4B81C9
:1060C0005C8185E293E021E234E0FC01659174910A
:1060D0004617570709F418C10C9628173907A9F76E
:1060E0006FCD2B813C8145E2E42E43E0F42E81E22A
:1060F00094E0F701459154912417350709F415C12F
:10610000FCE0EF0EF11C8E159F0599F7CC24CA9484
:10611000DC2C26C10E94AF14C9CDEB81E73008F01A
:10612000C5CDF0E0E356FB4C0C94DA338EE1ACAD18
:10613000BDAD1D928A95E9F788E089838A83A3CD56
:106140008C819AE0D92E7E01B1E2EB0EF11CF701B1
:106150002D2D11922A95E9F7B7010E94780D8983B8
:10616000F701DE01129601900D92DA94E1F79ECDCF
:10617000FC808AE0FE013596DE01919601900D9239
:106180008A95E1F789A19AA10E94BB079AA389A3E6
:106190008BA19CA10E94BB079CA38BA38DA19EA158
:1061A0000E94BB079EA38DA38FA198A50E94BB0749
:1061B00098A78FA337E08FEF3F1568F04AE0F49E71
:1061C000B001112464587D4F4AE050E0CE01819621
:1061D0000E945F3480E089830E94A30767CD6C81B1
:1061E0002AE0CE018196DC01E22F1D92EA95E9F7C3
:1061F000683008F047C0629FB001112464537D4F9E
:106200004AE050E00E940D3480E089838AE0FE017C
:10621000B196DE0112967ECEFC808AE0FE013596B4
:10622000DE01919601900D928A95E1F789A59AA5D4
:106230000E94BB079AA789A7F7E08FEFFF1568F0C8
:106240002AE0F29EB001112464537D4F4AE050E0F1
:10625000CE0181960E945F3480E089830E94760E91
:1062600025CD6C812AE0CE018196DC01E22F1D92C2
:10627000EA95E9F7683030F4629FB0011124645E5A
:106280007C4FBECF8FEFC1CFFC808AE0FE013596F8
:10629000DE01919601900D928A95E1F78BA19CA168
:1062A0000E94BB079CA38BA3F7E08FEFFF1568F05C
:1062B0002AE0F29EB0011124645E7C4F4AE050E077
:1062C000CE0181960E945F3480E089830E94F20DA6
:1062D000EDCC8091CF04882309F4A6C9E9BCD9BCD0
:1062E00009B400FEFDCF8091D8008F7D8093D80047
:1062F0008091E00082608093E0008091E00081FD69
:10630000FCCF0E94BF1190C9FC01369625913491B3
:106310002115310509F454CC4FE150E0BE016E5F08
:106320007F4FF90109958983C1CCF70138962591F2
:1063300034912115310509F4E9CE4CE150E0BE015C
:106340006B5F7F4FC701F90109956C01892B41F4FF
:10635000F7013A9685919491009711F0FC01099507
:10636000C982A4CC822B892B09F415CB12CB87E2EE
:1063700090E00E941D341B821C821D8220CE8CE383
:10638000669B02C08150E1F7669BFECF0895769828
:1063900080E48A95F1F7769A0895FC013AE03A95FF
:1063A000F1F798E020E080E031E040E24A95F1F733
:1063B000880F669B02C08160232742E04A95F1F76F
:1063C000000040E24A95F1F7915079F790E29A95F2
:1063D000F1F79CB132E03A95F1F7000040E24A95BE
:1063E000F1F796FB992790F992272081920F9083DD
:1063F0000895A1E0B0E0EFEFF1E30C948733198248
:106400008C017C01E60EF11C0E151F0541F481E0A4
:106410009981911180E02196E6E00C94A3330E94CB
:10642000BF31CE0101960E94CD31F80181938F01D9
:10643000EBCF6E9A769A08956E98769AEE9AEAE67F
:10644000F0E080818F7C808308956150770B91E02C
:1064500001C0990F6A95EAF720E031E0911108C078
:10646000222391F0769A80E48A95F1F77698089540
:10647000492F482339F0769A232740E44A95F1F7CB
:106480009695ECCF7698F9CF7698EDCFFF920F9353
:106490001F93CF93DF93EC018C01060F111DC017E2
:1064A000D10729F4CDB7DEB7E5E00C94A433F99019
:1064B0000E94C73168E08F2D0E942532F0CF1F92D5
:1064C0000F920FB60F9211240F931F932F933F93A8
:1064D0004F935F936F937F938F939F93AF93BF93EC
:1064E000EF93FF93CF93DF930F92CDB7DEB719826F
:1064F0000E94BF31CE0101960E94CD31082F069532
:1065000006950695282F22952570902F9570290FB6
:10651000922F937026952695920F982797708981D0
:10652000982B09F05CC0043008F059C080E28A95CD
:10653000F1F7769A6E9A82E08A95F1F700C0769824
:1065400088E0089F80011124D801AF5FBE4F1696E6
:10655000ED91FC9117973097A9F060918A017091A5
:106560008B0114962D913C911597260F371F11968C
:106570008D919C911297680F791F13964C911397E8
:106580008C910995F801EF5FFE4F6381662351F00E
:1065900020918A0130918B0184819581820F931F14
:1065A0000E9446320E94C73180E28A95F1F77698C0
:1065B0006E98769A80E28A95F1F7F801EF5FFE4FC8
:1065C0006081662351F020918A0130918B01818195
:1065D0009281820F931F0E94F9310E94BF310F9068
:1065E000DF91CF91FF91EF91BF91AF919F918F91EB
:1065F0007F916F915F914F913F912F911F910F91DB
:106600000F900FBE0F901F9018950F931F93CF936D
:10661000DF93EC0104970CF04CC0F8946E9A7698D6
:1066200085E08A95F1F700009C2F969595708C2F48
:106630008570980F892F83709695969523E0CC0FDF
:10664000DD1F2A95E1F7980F8E01092B0E94C731B3
:1066500000C068E0802F0E94253280E28A95F1F721
:106660006E98769A669B1EC087E090E066991CC083
:10667000FE01EF5FFE4F63816623F9F020918A01EE
:1066800030918B0184819581820F931F0E94F93193
:10669000811113C06E9A769A7894DF91CF911F91F1
:1066A0000F91089500C0DECF019729F46E9A769A73
:1066B000789480E0F2CF00C0D9CF0E94BF3180E44F
:1066C0008A95F1F776986E9A80E28A95F1F7CF5F16
:1066D000DE4F6881662351F020918A0130918B0151
:1066E00089819A81820F931F0E9446320E94C7318E
:1066F000789481E0D2CF2F923F924F925F926F9227
:106700007F928F929F92AF92BF92CF92DF92EF9241
:10671000FF920F931F93CF93DF93CDB7DEB7CA1BC2
:10672000DB0B0FB6F894DEBF0FBECDBF09942A88ED
:10673000398848885F846E847D848C849B84AA8495
:10674000B984C884DF80EE80FD800C811B81AA8122
:10675000B981CE0FD11D0FB6F894DEBF0FBECDBFED
:10676000ED010895AA1BBB1B51E107C0AA1FBB1F67
:10677000A617B70710F0A61BB70B881F991F5A95CD
:10678000A9F780959095BC01CD01089597FB072E40
:1067900016F4009407D077FD09D00E94B23307FCAD
:1067A00005D03EF4909581959F4F08957095619521
:1067B0007F4F0895EE0FFF1F0590F491E02D09948F
:1067C0006927962769277827872778270895FB0167
:1067D000DC0102C005900D9241505040D8F7089559
:1067E000FB01DC0104C08D910190801921F441501E
:1067F0005040C8F7881B990B0895FB01DC0102C0CB
:1068000001900D9241505040D8F70895DC0101C02D
:106810006D9341505040E0F70895DC01CB01FC013D
:10682000F999FECF06C0F2BDE1BDF89A319600B4E9
:106830000D9241505040B8F70895F999FECF92BD9E
:1068400081BDF89A992780B50895A8E1B0E042E0AB
:1068500050E00C940F34DC01A40FB51F41505040A0
:1068600048F0CB01840F951F2E910E943C3441507B
:106870005040D0F70895262FF999FECF92BD81BDE3
:10688000F89A019700B4021639F01FBA20BD0FB66E
:10689000F894FA9AF99A0FBE08950396272F0E944A
:1068A0003C340E943B34252F0E943C34242F0C940E
:1068B0003C340196272F0E943C340C943B34DC017D
:1068C000CB0103C02D910E946A3441505040D0F753
:1068D0000895262FF999FECF1FBA92BD81BD20BD24
:1068E0000FB6F894FA9AF99A0FBE01960895F894A3
:1068F000FFCFC712EF129D14EF129D142213431302
:106900009D144C145914EB1CEB1C201D201DE91D7B
:10691000051E461D461D0A1E771E881E881E752FE1
:106920008F2F952F562E562ECF2FE12FF42F32304A
:1069300037305F3071308A308D309630A030B830CB
:08694000EF300C31313144311C
:106948000100000001000000000000000501000037
:10695800000406000000000000F5F6F73133323677
:10696800919094669701BB04AC0BBA04A50B9E0BDF
:1069780050011401AF0001011E0A280801919094EA
:106988006697323331F7F6F53698CC693A4B2DDFF6
:10699800EA818283E200E900EA00B500B600B700A8
:1069A800CD008301CC008A019201940121022302C7
:1069B80024022502260227022A02B300B4006F002F
:1069C80070009F01CB019F02A002F20144227B4983
:0C69D800012701AC00BF04D804F8040043
:00000001FF
